:020000040800F2
:1000000000070020F1010008BD2C0008752C000835
:100010009D2C0008752C0008952C0008F3010008A1
:10002000F3010008F3010008F3010008B13C0008E7
:10003000F3010008F3010008F3010008F3010008D0
:10004000F3010008F3010008F3010008F3010008C0
:10005000F3010008F301000829680008516800084E
:1000600079680008A1680008C9680008F301000861
:10007000F3010008F3010008F3010008F301000890
:10008000F3010008F3010008F3010008292C00081F
:10009000552C0008652C0008F3010008F1680008E1
:1000A000F3010008F3010008F3010008F301000860
:1000B000D9690008F3010008F3010008F301000802
:1000C000F3010008F3010008F3010008F301000840
:1000D000F3010008F3010008C5690008F3010008F6
:1000E00055690008F3010008F3010008F301000856
:1000F000F3010008F3010008F3010008F301000810
:10010000F3010008F3010008F3010008F3010008FF
:10011000F3010008F3010008F3010008F3010008EF
:10012000F3010008F3010008F3010008F3010008DF
:10013000F3010008F3010008F3010008F3010008CF
:10014000F3010008F3010008F3010008195E00083C
:10015000F3010008F3010008F3010008F3010008AF
:10016000F3010008F3010008F3010008F30100089F
:10017000F3010008F3010008F3010008F30100088F
:10018000F3010008F3010008F3010008F30100087F
:10019000F3010008F3010008F3010008F30100086F
:1001A000F3010008F3010008F3010008F30100085F
:1001B000F3010008F3010008F3010008F30100084F
:1001C000F3010008F3010008F3010008F30100083F
:1001D000F3010008F3010008F3010008F30100082F
:1001E0009D15000800000000000000000000000055
:1001F00002E000F000F8FEE772B6374880F30888A6
:10020000364880F3098836483649086040F20000D5
:10021000CCF200004EF63471CEF200010860BFF35C
:100220004F8FBFF36F8F40F20000C0F2F0004EF628
:100230008851CEF200010860BFF34F8FBFF36F8F7C
:100240004FF00000E1EE100A4EF63C71CEF20001D4
:100250000860062080F31488BFF36F8F05F0A4FABE
:1002600006F088F94FF055301F491B4A91423CBFB8
:1002700041F8040BFAE71D49184A91423CBF41F886
:10028000040BFAE71A491B4A1B4B9A423EBF51F82E
:10029000040B42F8040BF8E700201849184A914271
:1002A0003CBF41F8040BFAE705F082FA06F0B6F914
:1002B000144C154DAC4203DA54F8041B8847F9E797
:1002C00000F042F8114C124DAC4203DA54F8041B12
:1002D0008847F9E705F06ABA0007002000230020EC
:1002E0000000000808ED00E00001002000070020E9
:1002F0003070000800230020BC230020C023002011
:1003000004590020E0010008E4010008E4010008AD
:10031000E40100082DE9F04F2DED108AC1F80CD052
:10032000C3689D46BDEC108ABDE8F08F002383F3BF
:1003300011882846A047002004F01CFDFEE704F0C9
:100340009BFC00DFFEE70000F8B501F0A3F905F023
:10035000CDF930B12A4B00220F211A725A729972CC
:10036000DA7205F0A5F9074605F00AFA05460028F5
:100370003AD1244B9F4237D001339F4237D0224B92
:1003800027F0FF029A4235D1F8B200F025FF2E4641
:1003900042F2107400F026FF08B10024264601F056
:1003A00069FD20B1032000F085F80024264635B110
:1003B000164B9F4203D005F0DBF9002426460020AF
:1003C00005F080F9124B1B6913F4807316D00EB13F
:1003D00000F086F801F0CCFA00F070FF204600F043
:1003E000E5F800F07DF8F9E72E460024D2E7044650
:1003F0000126CFE7064641F28834CBE71C46E9E701
:1004000000230020010007B0000008B0263A09B020
:100410000004024008B501F009F9A0F12003584298
:10042000584108BD07B541F21203022101A8ADF8F9
:10043000043001F019F903B05DF804FB38B530233E
:1004400083F31188174803680BB104F05FFD164A67
:10045000144800234FF47A7104F04EFD002383F317
:100460001188124C236813B12368013B2360636831
:1004700013B16368013B63600D4D2B7833B963683A
:100480007BB9022001F0D6F9322363602B78032B6D
:1004900007D163682BB9022001F0CCF94FF47A73CD
:1004A000636038BDC02300203D040008E024002024
:1004B000D8230020084B187003280CD8DFE800F080
:1004C00008050208022001F0A5B9022001F094B944
:1004D000024B00225A607047D8230020E0240020FD
:1004E00010B501F0C7FC30B1294B03221A70294B1B
:1004F00000225A6010BD284B284A1C461968013159
:10050000F8D004339342F9D16268254B9A42F1D96D
:10051000244B9B6803F1006303F580339A42E9D2D0
:1005200005F0FAF805F00CF9002001F0CDF80220F2
:10053000FFF7C0FF1C4B1A6C00221A64196E1A6672
:10054000196E596C5A64596E5A665A6E5A6942F05D
:1005500080025A615A6922F080025A615A691A6906
:1005600042F000521A611A6922F000521A611B69A6
:1005700072B64FF0E0233021C3F8084DD4E90032C1
:1005800081F311889D4683F308881047B2E700BFC6
:10059000D8230020E02400200000010820000108EA
:1005A000FFFF000800230020003802402DE9F04F33
:1005B00093B0AC4B00902022FF210AA89D6801F067
:1005C00081F9A94A1378A3B9A848012103601170E1
:1005D000302383F3118803680BB104F097FCA44A1D
:1005E000A24800234FF47A7104F086FC002383F3C1
:1005F0001188009B13B19F4B009A1A609E4A009C81
:100600001378032B1EBF002313709A4A4FF0000A81
:1006100018BF5360D3465646D146012001F0FAF880
:1006200024B1944B1B68002B00F01582002000F0D1
:10063000FDFF0390039B002B01DA00F087FE039B74
:10064000002BEDDB012001F0D7F8039B213B162B9B
:10065000E3D801A252F823F0B5060008DD06000831
:10066000710700081B0600081B0600081B0600088F
:10067000FB070008CB090008E50800084709000847
:100680006F090008950900081B060008A709000863
:100690001B060008190A0008550700081B06000879
:1006A0005D0A0008C1060008550700081B0600087F
:1006B000470900080220FFF7ADFE002840F0F58151
:1006C000009B0221BAF1000F08BF1C4605A841F2A9
:1006D0001233ADF8143000F0C7FF9EE74FF47A7084
:1006E00000F0A4FF071EEBDB0220FFF793FE0028BB
:1006F000E6D0013F052F00F2DA81DFE807F0030AB8
:100700000D10133605230593042105A800F0ACFF56
:1007100017E054480421F9E758480421F6E75848FF
:100720000421F3E74FF01C08404600F0CFFF08F12A
:1007300004080590042105A800F096FFB8F12C0FDD
:10074000F2D1012000FA07F747EA0B0B5FFA8BFBA7
:100750004FF0000901F002F926B10BF00B030B2B4F
:1007600008BF0024FFF75EFE57E746480421CDE7A7
:10077000002EA5D00BF00B030B2BA1D10220FFF70D
:1007800049FE074600289BD0012000F09DFF022073
:10079000FFF790FE00261FFA86F8404600F0A4FFFF
:1007A000044690B10021404600F0B6FF0136002813
:1007B000F1D1BA46044641F21213022105A8ADF860
:1007C00014303E4600F050FF27E70120FFF772FE8D
:1007D0002546244B9B68AB4207D9284600F076FF9C
:1007E000013040F067810435F3E7234B00251D708D
:1007F000204BBA465D603E46ACE7002E3FF460AF4A
:100800000BF00B030B2B7FF45BAF0220FFF752FEC4
:10081000322000F00BFFB0F10008FFF651AF18F0E6
:1008200003077FF44DAF0F4A926808EB050393422C
:100830003FF646AFB8F5807F3FF742AF124B0193CA
:10084000B84523DD4FF47A7000F0F0FE0390039A70
:10085000002AFFF635AF019B039A03F8012B0137FD
:10086000EDE700BF00230020DC240020C02300208F
:100870003D040008E0240020D823002004230020A9
:10088000082300200C230020DC230020C820FFF7D1
:10089000C1FD074600283FF413AF1F2D11D8C5F145
:1008A000200242450AAB25F0030028BF4246834997
:1008B0000192184400F0E0FF019A8048FF2101F006
:1008C00001F84FEAA8037D490193C8F3870228463F
:1008D00001F000F8064600283FF46DAF019B05EBE0
:1008E000830537E70220FFF795FD00283FF4E8AEC7
:1008F00000F032FF00283FF4E3AE0027B846704B0B
:100900009B68BB4218D91F2F11D80A9B01330ED008
:1009100027F0030312AA134453F8203C05934046E2
:10092000042205A901F05EFA04378046E7E738465D
:1009300000F0CCFE0590F2E7CDF81480042105A864
:1009400000F092FE06E70023642104A8049300F05F
:1009500081FE00287FF4B4AE0220FFF75BFD002883
:100960003FF4AEAE049800F0DFFE0590E6E700230A
:10097000642104A8049300F06DFE00287FF4A0AE6B
:100980000220FFF747FD00283FF49AAE049800F0DC
:10099000DBFEEAE70220FFF73DFD00283FF490AEC2
:1009A00000F0EAFEE1E70220FFF734FD00283FF403
:1009B00087AE05A9142000F0E5FE04210746049047
:1009C00004A800F051FE3946B9E7322000F02EFEAF
:1009D000071EFFF675AEBB077FF472AE384A926809
:1009E00007EB090393423FF66BAE0220FFF712FDBF
:1009F00000283FF465AE27F003074F44B9453FF4A4
:100A0000A9AE484600F062FE0421059005A800F05A
:100A10002BFE09F10409F1E74FF47A70FFF7FAFCB5
:100A200000283FF44DAE00F097FE002844D00A9B0A
:100A300001330BD008220AA9002000F04BFF002848
:100A40003AD02022FF210AA800F03CFFFFF7EAFC81
:100A50001C4804F095F913B0BDE8F08F002E3FF468
:100A60002FAE0BF00B030B2B7FF42AAE0023642177
:100A700005A8059300F0EEFD074600287FF420AEA0
:100A80000220FFF7C7FC804600283FF419AEFFF7AD
:100A9000C9FC41F2883004F073F9059800F0A2FF18
:100AA000464600F05BFF3C46B7E5064652E64FF08F
:100AB000000905E6BA467EE637467CE6DC230020E0
:100AC00000230020A0860100094A136849F269004A
:100AD00099B21B0C00FB01331360064B186844F2FB
:100AE000506182B2000C01FB0200186080B27047B6
:100AF000182300201423002010B5002110220446E2
:100B000000F0E0FE034B03CB206061601868A0603A
:100B100010BD00BF107AFF1F2DE9F041ADF5507DEB
:100B20000DF13C086EAC40F2751207460D4610A858
:100B30000021C8F8001000F0C5FE4FF4C472002177
:100B4000204600F0BFFE02F0C1F8274B4FF47A7246
:100B5000B0FBF2F0186093E80700022384E8070076
:100B60000DF5ED702382FFF7C7FF47F605231F49F8
:100B7000238407A806F046F81D2384F832310DF2CD
:100B8000EB2207AB0DF1340C1E4603CE6645106018
:100B90005160334602F10802F6D1306810603379B3
:100BA000137141460122204600F03EFF00230393CB
:100BB000AB7E029305F11903019380B20123CDE9C5
:100BC00004800093E97E06A3D3E90023384602F0AF
:100BD00045FC0DF5507DBDE8F08100BFAFF300800E
:100BE0009E6AC421818A46EEE8240020146C000825
:100BF0002DE9F0412C4C237ADAB080460D465BBBE0
:100C000027A9284601F020F80746002842D19DF880
:100C10009D60C82E3ED801464FF4A662204600F0E3
:100C200051FE4FF48073C4F8F8314FF40073C4F8E8
:100C30000C334FF44073C4F8203432460DF19E015A
:100C400004F1090000F018FE26449DF89C307772EC
:100C500023720BB9EB7E23728122002106AC27A8F8
:100C600000F030FE0122214627A801F029F80023D8
:100C70000393AB7E029305F1190380B201932823FD
:100C8000CDE904400093E97E05A3D3E90023404663
:100C900002F0E4FB5AB0BDE8F08100BFAFF3008082
:100CA00026417272DF25D7B708460020F0B5254EE1
:100CB0004FF48A7505FB0065F1B096F8D83085F8D9
:100CC000DC300024D822214685F8E8403AA800F01C
:100CD000F9FD06F1090000F0EDFDD5F8E4308DF8DE
:100CE000F000C2B206AF06F109010DF1F100CDE945
:100CF0003A3400F0C1FD394601223AA801F00CF85F
:100D000080B2CDE9047008230127CDE9023706F14E
:100D1000D803019330230093317A0B4807A3D3E91A
:100D2000002302F09BFBA04206DD01F0CFFFC5F8D7
:100D3000E000384671B0F0BD2046FBE778F6339FFF
:100D400093CACD8D08460020003500202DE9F041E2
:100D50001D4D1E4E1E4F86B0284602F0ABFB0346CB
:100D600058B30024CDE90344ADF81440027B8DF85C
:100D7000142099684068029403AA03C21B68DFF834
:100D8000548043F00043029301F0A2FF821941F125
:100D90000003009402A9384601F04AFAA04205DD9A
:100DA000284602F08BFB88F80040D5E798F8003021
:100DB000072B05D8013388F8003006B0BDE8F08174
:100DC000014802F07BFBF8E70035002040420F00AD
:100DD000303500203D4B002070B50D4614461E46B0
:100DE00002F098FA50B9022E10D1012C0ED112A3A4
:100DF000D3E90023C5E90023012007E0282C10D007
:100E000005D8012C09D0052C0FD0002070BD302C46
:100E1000FBD10BA3D3E90023ECE70BA3D3E9002319
:100E2000E8E70BA3D3E90023E4E70BA3D3E900230E
:100E3000E0E700BFAFF30080401DA12026812A0B10
:100E400078F6339F93CACD8D9E6AC421818A46EE7F
:100E500026417272DF25D7B7F017304A39059E5602
:100E600038B505460E4C0021013500F055FCA4F8BC
:100E70002C55B4F82C0500F037FC78B1B4F82C05EB
:100E800000F042FC014648B9B4F82C0500F044FCDF
:100E9000B4F82C350133A4F82C35EAE738BD00BF8F
:100EA0000846002010B50A4B0A4A1A6003F5805321
:100EB00093F860203AB9DC6D2CB1204601F058F867
:100EC000204605F0DFFDBDE81040034801F050B8B2
:100ED00030350020D06C0008784500202DE9F04F17
:100EE0008FB000AF05460C4602F014FA002849D135
:100EF000237E022B1BD1E38A012B18D101F0E6FEE1
:100F00000646FFF7E1FD03464FF4C870DFF8C482E0
:100F1000B3FBF0F206F5167602FB103316FA83F3F4
:100F2000C8F80030E37E33B9A34B00221A703C3777
:100F3000BD46BDE8F08F07F12401204600F042FED7
:100F40000028F4D107F11400FFF7D6FD97F82640EA
:100F500007F11401224607F1270005F0DDFD002806
:100F6000E2D10F2C08D8944B1C70D8F80030A3F5B0
:100F70001673C8F80030DAE797F82410284602F014
:100F8000C1F9D4E7E38A282B2BD010D8012B23D02A
:100F9000052BCCD1BFF34F8F8849894BCA6802F427
:100FA000E0621343CB60BFF34F8F00BFFDE7302BF0
:100FB000BDD1844EE17E327A9142B8D1607E314615
:100FC000002291F8DC50854200F0A5800132042A0D
:100FD00001F58A71F5D1AAE721462846FFF79CFD65
:100FE000A5E721462846FFF703FEA0E7B2F8EC503C
:100FF0007B6005F103094FEA99094FEA8902D11D87
:10100000C908A8EBC1039D46EB460021584600F0F5
:1010100059FC04F1EE012A463144584600F02CFCFC
:101020007B6813B9012000F04FFB96F8D20000F066
:101030005BFB044630B9307200F08EFB204600F0B6
:1010400043FBB1E0D6F8D4203AB996F8D200B6F80E
:101050002C25824201D8FFF703FFD6F8D4202A447A
:10106000944208D296F8D200B6F82C25013082427C
:1010700001D8FFF7F5FE70685FFA89F2594600F073
:1010800029FC08B9C54679E0726896F8D2002A446E
:101090007260D6F8D42005EB0209C6F8D49000F0AF
:1010A00023FB814509D396F8D220D6F8D40001322B
:1010B000001B86F8D220C6F8D400FF2D0FD80024DC
:1010C000347200F049FB204600F0FEFA00F0D2FE38
:1010D0003D4B188108B9FFF703FAC54627E7BB68FF
:1010E00096F8D9000AFB0362FB68D2F8E41082F894
:1010F000E83001F58061C2F8E030C2F8E410FFF793
:10110000D5FDFFF723FE96F8D920013202F0030245
:1011100086F8D920B6E74FF48A7A0AFB02F505F182
:10112000EA013144204600F023FEF86000287FF4F5
:10113000FEAE3544012285F8E82001F0C7FDD5F860
:10114000E020D6ED007ADFED216A801A192838BF39
:10115000192040F6B832904228BF1046B8EE677AA0
:1011600007EE900AF8EEE77A67EEA67ADFED186AE6
:10117000E7EE267AFCEEE77AC6ED007A96F8D930EB
:10118000BB60BA6873680AFB02F4321992F8E8107F
:1011900059B1D2F8E4108B42E8463FF427AF002162
:1011A00082F8E810C2F8E010C5467368064A9B0A48
:1011B00001331381BBE600BFF934002000ED00E0ED
:1011C0000400FA0508460020E8240020CDCCCC3DE0
:1011D0006666663FFC340020014B1870704700BF04
:1011E000F424002030B54FF000542B4B22689A4273
:1011F00085B007D004F0CEFA044620BB0024204678
:1012000005B030BD254B627D25481A70237D0372E1
:101210004FF48073C0F8F8314FF40073C0F80C330A
:1012200000254FF44073C0F820341E49C0F8E45044
:10123000C922093000F020FB2046E022294600F0B8
:1012400041FB0124DBE7184A184D136C43F000738F
:101250001364AA6D164B9A42D0D12B6E013B7E2BA4
:10126000CCD8144A07CA01AB83E80700184603210B
:1012700000F0CEFD6B6D83424FF00003BED12A6DAE
:101280008A4201BFAB65054B2A6E1A7003BF0A4B39
:10129000EA6D1A601C46B2E79AAD44C5F4240020FA
:1012A000084600201600002000380240006600407A
:1012B0005041A0B0586600401023002037B51A4DA9
:1012C00000F0D8FD02236B71184B2881196818486B
:1012D000012201F097FB00230193164B164900935E
:1012E0001648174B4FF4805201F0E4FF154B197864
:1012F00011B1124802F006F801F0E8FC0446FFF7CD
:10130000E3FB4FF4C873B0FBF3F202FB130304F5E5
:10131000167010FA83F00C4B186004F031FA08B123
:101320000F232B8103B030BDE824002010230020C0
:1013300030350020D90D0008F824002000350020A9
:10134000DD0E0008F4240020FC3400202DE9F04FCD
:101350002DED028B0FF23829D9E90089834C93B027
:101360000BAE9FED7E8BFFF7F1FC814FDFF828A2DB
:1013700000230A93ADF834300B9373604FF0000BE9
:101380005B468DED008B01250DF11D0207A9384646
:101390008DF81C508DF81DB001F0E2FA9DF81C305C
:1013A000002B40F0A580204601F0B4FF064600283F
:1013B00045D1704F01F08AFC3B6898423FD301F061
:1013C00085FC8246FFF780FB4FF4C873B0FBF3F255
:1013D00002FB13030AF5167010FA83F03860664FAB
:1013E00097F800B0CBF1100ABBF1000F14BF3346E1
:1013F0002B465FFA8AFA0EA88DF82830FFF77CFB9F
:10140000BAF1060F28BF4FF0060A0EAB03EB0B0133
:1014100052460DF1290000F02FFA0AAB039318236E
:1014200002930AF10102554BD2B2CDE90053049266
:1014300020464CA3D3E9002301F0B2FF3E7001F037
:1014400045FC4F4A4F4D1368C31AB3F57A7F2ED32C
:10145000106001F03DFC02460B46204602F038F8D1
:10146000204601F057FF10B32B7A474E002B14BFD4
:1014700003230223737101F029FC0EAF4FF47A733A
:101480000122B0FBF3F039463060304600F072FBC9
:10149000182302933D4B019380B240F25513CDE9DE
:1014A0000370009342464B46204601F079FF2B7AA9
:1014B00093B101F00BFC002607464FF48A7A95F8A9
:1014C000D900304400F003000AFB005393F8E820F1
:1014D00092B30136042EF2D1C82003F051FC2B7ACE
:1014E000002B7FF43DAF13B0BDEC028BBDE8F08F55
:1014F000DAF8143083F00203CAF814305946102287
:101500000EA800F0DFF90DF11E0308AA0AA938465B
:1015100000F08EFF96E803000FAB83E803009DF810
:1015200034308DF844300A9B0E930EA9DDE9082370
:10153000204602F0A1F921E7D3F8E02042B12B6860
:10154000FA2B38BFFA23BA1A0533B2EB430FC0D3D4
:10155000FFF7ACFB0028BCD1BEE700BF00000000D5
:1015600000000000401DA12026812A0B003500202C
:1015700030350020FC340020F9340020F8340020FD
:10158000384B002008460020E82400203C4B002077
:10159000F1C6A7C1D068080F0004024008B505488D
:1015A00000F0E2FFBDE80840034A0449002005F0CE
:1015B00063BA00BF303500208C4B0020A50E000818
:1015C0002DE9F84F4FF47A73DFF85880DFF8589020
:1015D00006460D4602FB03F7002498F900305A1C1A
:1015E0005FFA84FA01D0A34212D159F824000368AB
:1015F0002A46D3F820B031463B46D847854207D12A
:10160000074B012083F800A0BDE8F88F0124E4E730
:10161000002CFBD04FF4FA7003F0B2FB0020F3E78C
:10162000804B00201C2300202023002007B500232E
:10163000024601210DF107008DF80730FFF7C0FFCA
:1016400020B19DF8070003B05DF804FB4FF0FF30B8
:10165000F9E700000A4608B50421FFF7B1FF80F062
:101660000100C0B2404208BD30B4074B0A461978A9
:10167000064B53F821402368DD69054B0146AC4613
:10168000204630BC604700BF804B00202023002054
:10169000A086010070B503F0A5FE094E094D30800B
:1016A000002428683388834208D903F095FE2B680C
:1016B00004440133B4F5803F2B60F2D370BD00BF0A
:1016C000824B0020404B002003F042BF00F100603D
:1016D00000F580300068704700F10060920000F56E
:1016E000803003F0CDBE0000054B1A68054B1B8807
:1016F0009B1A834202D9104403F06EBE002070474B
:10170000404B0020824B0020024B1B68184403F022
:101710006BBE00BF404B0020024B1B68184403F017
:101720007BBE00BF404B002010F003030AD1B0F590
:10173000047F05D200F10050A0F51040D0F8003829
:10174000184670470023FBE700F10050A0F5104059
:10175000D0F8100A70470000064991F8243033B1E0
:101760000023086A81F824300822FFF7B5BF012062
:10177000704700BF444B0020014B1868704700BF02
:10178000002004E070B5194B1D68194B0138C5F3F2
:101790000B0408442D0C04221E88A6420BD15C6861
:1017A0000A46013C824213460FD214F9016F4EB132
:1017B00002F8016BF6E7013A03F10803ECD181422C
:1017C0000B4602D22C2203F8012B0A4A0524168864
:1017D000AE4204D1984284BF967803F8016B013C75
:1017E00002F10402F3D1581A70BD00BF002004E0DA
:1017F000746C0008606C0008022802D1044B9861E8
:101800007047012802BF024B08229A61704700BF4F
:1018100000040240022804D1054B4FF400329A61C3
:1018200070470128FCD1024B4FF40022F7E700BFBC
:1018300000040240022805D1064A536983F00203DE
:10184000536170470128FCD1024A536983F00803B1
:10185000F6E700BF0004024070B504464FF47A7604
:101860004CB1412C254628BF412506FB05F003F06D
:1018700087FA641BF4E770BD10B50023934203D0D0
:10188000CC5CC4540133F9E710BD000010B5013839
:1018900010F9013F3BB191F900409C4203D11AB1CC
:1018A0000131013AF4E71AB191F90020981A10BDFC
:1018B0001046FCE703460246D01A12F9011B002924
:1018C000FAD1704702440346934202D003F8011B49
:1018D000FAE770472DE9F8431F4D144695F8242088
:1018E0000746884652BBDFF870909CB395F82430C9
:1018F0002BB92022FF2148462F62FFF7E3FF95F81E
:101900002400C0F10802A24228BF2246D6B24146B6
:10191000920005EB8000FFF7AFFF95F82430A41B81
:101920001E44F6B2082E17449044E4B285F82460B1
:10193000DBD1FFF711FF0028D7D108E02B6A03EBBA
:1019400082038342CFD0FFF707FF0028CBD10020CE
:10195000BDE8F8830120FBE7444B0020024B1A78D6
:10196000024B1A70704700BF804B00201C230020E0
:1019700038B5174C174D204602F058FD2946204631
:1019800002F080FD2D686A6D936B23F4002393634E
:101990004FF47A70FFF760FF0F49284602F078FE97
:1019A0006A6D0E4D936B28680D4943F400239363D1
:1019B000A0424FF4E1330B6001D002F097FC68685D
:1019C000A04204D0BDE83840054902F08FBC38BDC4
:1019D00070500020F86D0008006E000820230020E1
:1019E0006C4B002070B50C4B0C4D1E780C4B55F811
:1019F00026209A4204460DD00A4B00211422184694
:101A0000FFF760FF0460014655F82600BDE870400E
:101A100002F06CBC70BD00BF804B00202023002072
:101A2000705000206C4B00202DE9F0470D46044615
:101A300000219046284640F27912FFF743FF2346E3
:101A400020220021284601F0B9FE231D0222202178
:101A5000284601F0B3FE631D03222221284601F02F
:101A6000ADFEA31D03222521284601F0A7FE04F1A7
:101A7000080310222821284601F0A0FE04F11003DB
:101A800008223821284601F099FE04F111030822AA
:101A90004021284601F092FE04F112030822482159
:101AA000284601F08BFE04F1140320225021284621
:101AB00001F084FE04F1180340227021284601F051
:101AC0007DFE04F120030822B021284601F076FEB5
:101AD00004F121030822B821284601F06FFE04F129
:101AE0002207C0263B46314608222846083601F028
:101AF00065FEB6F5A07F07F10107F3D104F13203CB
:101B000008223146284601F059FE002704F1330A25
:101B100094F832304FEAC7099F4209F5A47615D3ED
:101B2000B8F1000F08D1314604F599730722284611
:101B300001F044FE09F24F16274694F832213B1B70
:101B400093420CD3F01DC008BDE8F0870AEB0703F1
:101B500008223146284601F031FE0137D8E707F266
:101B6000331331460822284601F028FE0836013793
:101B7000E3E7000013B50446084600210160234650
:101B8000C0F803102022019001F018FE0198231DD7
:101B90000222202101F012FE0198631D032222215E
:101BA00001F00CFE0198A31D0322252101F006FE81
:101BB000019804F108031022282101F0FFFD0720FD
:101BC00002B010BDF7B50023047F00910E46072236
:101BD0001946054601F0B6FC731C00930122002350
:101BE0000721284601F0AEFCC4B9B31C00930522BE
:101BF00023460821284601F0A5FC0D243746B2787B
:101C0000BB1B934211D32B7FA88A0734E408BBB9CE
:101C1000844294BF0020012003B0F0BDAB8ADB00FA
:101C2000083BDB08B3700824E8E7FB1C009321465F
:101C300000230822284601F085FC08340137DEE73E
:101C4000201A18BF0120E7E7F7B50023047F0091B1
:101C50000E4608221946054601F074FC731CC4B9EF
:101C60000822009311462346284601F06BFC1024FD
:101C7000012372785F1C013B934211D32B7FA88A0A
:101C80000734E408BBB9844294BF0020012003B0AC
:101C9000F0BDAB8ADB00083BDB0873700824E7E784
:101CA000F3190093214600230822284601F04AFC3C
:101CB00008343B46DDE7201A18BF0120E7E70000A3
:101CC000F8B50E4605461446002181223046FFF73E
:101CD000F9FD2B4608220021304601F06FFD7CB94A
:101CE0006B1C07220821304601F068FD0F240123F8
:101CF0006A785F1C013B934204D3E01DC008F8BD25
:101D00000824F4E7EB1921460822304601F056FD7D
:101D100008343B46ECE70000F8B50E46054614468D
:101D20000021CE223046FFF7CDFD2B462822002190
:101D3000304601F043FD7CB905F108030822282153
:101D4000304601F03BFD30242F462A7A7B1B93421C
:101D500004D3E01DC008F8BD2824F5E707F1090306
:101D600021460822304601F029FD08340137ECE70E
:101D7000F7B5047F00910E4601231022002105468D
:101D800001F0E0FBC4B9B31C0093092223461021E3
:101D9000284601F0D7FB192437467288BB1B9A42AC
:101DA00011D82B7FA88A0734E408BBB9844294BFBA
:101DB0000020012003B0F0BDAB8ADB00103BDB0844
:101DC00073801024E8E73B1D00932146002308227E
:101DD000284601F0B7FB08340137DEE7201A18BFA8
:101DE0000120E7E730B5094D0A4491420DD011F8C2
:101DF000013B5840082340F30004013B2C4013F002
:101E0000FF0384EA5000F6D1EFE730BD2083B8ED40
:101E1000F7B54FF0FF33DFF854C0DFF854E000EBC4
:101E200081011A4688421CD050F8044B019401AF3E
:101E3000042417F8015B82EA05620825DB181646C0
:101E400005F1FF355241002EBCBF83EA0C0382EA44
:101E50000E0215F0FF05F1D1013C14F0FF04E8D1AA
:101E6000E0E7D843D14303B0F0BD00BF9336EAA901
:101E7000EBE1F042F7B5384A106851686B4603C38E
:101E80006A4636493648082304F056FE04460028C0
:101E900033D10A25334A106851686B4603C36A463A
:101EA00031492F48082304F047FE0446002849D052
:101EB0000369B3F5F81F45D8B0F8661040F27A52BE
:101EC00091423FD1294A024402F15C018B4239D34D
:101ED0005C3B234900209E1AFFF784FF32460746E9
:101EE00004F164010020FFF77DFFA3689F4229D120
:101EF000E368984208BF002524E00369B3F5F81FA2
:101F000027D8418B40F27A52914220D1174A02449D
:101F100002F110018B4218D3103B114900209D1A89
:101F2000FFF760FF2A46064604F118010020FFF77C
:101F300059FFA3689E4202D1E368984201D00D2563
:101F4000A8E70025284603B0F0BD1025A2E70C2520
:101F5000A0E70B259EE700BF946C0008DCFF1E0085
:101F6000000001089D6C000890FF1E000800FFF7AC
:101F700010B5037C044613B9006804F0C5FD204683
:101F800010BD00000023BFF35B8FC360BFF35B8F06
:101F9000BFF35B8F8360BFF35B8F7047BFF35B8FD3
:101FA0000068BFF35B8F704770B505460C30FFF7D4
:101FB000F5FF05F1080604463046FFF7EFFFA042A3
:101FC00006D930466D68FFF7E9FF2544281A70BD31
:101FD0003046FFF7E3FF201AF9E7000070B5054629
:101FE000406898B105F10800FFF7D8FF05F10C062D
:101FF00004463046FFF7D2FF8442304694BF6D68F6
:102000000025FFF7CBFF013C2C44201A70BD0000D7
:1020100038B50C460546FFF7C7FFA04210D305F1BF
:102020000800FFF7BBFF04446868B4FBF0F100FB55
:102030001144BFF35B8F0120AC60BFF35B8F38BDF1
:102040000020FCE72DE9F041144607460D46FFF756
:10205000C5FF844228BF0446D4B1B84658F80C6B7B
:102060004046FFF79BFF3044286040467E68FFF7FC
:1020700095FF331A9C4203D86C600120BDE8F081C3
:102080006B60A41B3B68AB602044E8600220F5E76E
:102090002046F3E738B50C460546FFF79FFFA04200
:1020A00010D305F10C00FFF779FF04446868B4FB16
:1020B000F0F100FB1144BFF35B8F0120EC60BFF334
:1020C0005B8F38BD0020FCE72DE9FF41884669465B
:1020D0000746FFF7B7FF6C4606B204EBC6060025BD
:1020E000B44209D06268206808EB0501FFF7C4FB21
:1020F000636808341D44F3E729463846FFF7CAFFF2
:10210000284604B0BDE8F081F8B505460C300F460E
:10211000FFF744FF05F1080604463046FFF73EFF8F
:10212000A042304688BF6C68FFF738FF201A38603D
:1021300020B130462C68FFF731FF2044F8BD000085
:1021400073B5144606460D46FFF72EFF844228BF9E
:1021500004460190DCB101A93046FFF7D5FF019B91
:1021600033B93268C5E90233C5E9002401200CE027
:102170009C4238BF01942860019868608442F5D978
:102180003368AB60241AEC60022002B070BD2046B8
:10219000FBE700002DE9FF410F466946FFF7D0FF3E
:1021A0006C4600B204EBC0050026AC4209D0D4F85E
:1021B000048054F8081BB8194246FFF75DFB4644FB
:1021C000F3E7304604B0BDE8F081000038B50546BD
:1021D000FFF7E0FF044601462846FFF719FF2046B7
:1021E00038BD000010B4026854681A4623465DF8F2
:1021F000044B1847002070470020704770470000CC
:10220000002070470E20704700F5805090F8C800FD
:10221000C0F340007047000000F5805090F9D000F6
:102220007047000000F58050C0F8CC1001207047C6
:10223000F7B50C68BDF8207014F0005470D10D7B18
:10224000082D6DD8302585F311884569AE68760173
:102250000CD4AC68240108D4AC6814F080545DD16F
:1022600084F31188204603B0F0BD01240E6804F108
:10227000180C002EB8BFF6004FEA0C1CB4BF46F095
:102280000406760545F80C600E680FFA84FC16F01B
:10229000804F18BF05EB0C1E05EB0C1C1EBFDEF8B3
:1022A000806146F00206CEF880610E7BCCF8846136
:1022B00005EB04158E68C5F88C614E68C5F8886119
:1022C000DCF8805145F00105CCF8805100EB441654
:1022D00041F268052E4405EB44150544C6E9002388
:1022E00008350E4601F10C0C56F804EB45F804EBEA
:1022F0006645F9D1843436882E8000EB441407F00B
:102300000305267926F00B0635432571002484F356
:102310001188009700F0FCFC0120A4E70224A5E747
:102320004FF0FF309FE7000013B500F58054019196
:10233000E06DFFF753FE1F280AD90199E06D2022B6
:10234000FFF7C2FEA0F120035842584102B010BD71
:102350000020FBE708B5302383F3118800F5805097
:10236000C06DFFF70FFE002383F3118808BD000046
:1023700000220260828142608260704710B50022B4
:102380000023C0E900230023044603810C30FFF73B
:10239000EFFF204610BD0000F0B5054600F5805067
:1023A0000C4690F8C83013F0040FC3F3800108BF47
:1023B000114661F3820304F1840680F8C83005EB0E
:1023C000461389B01B79D8072ED57AB319072DD4B7
:1023D0006846FFF7D3FF05EB441303F5835303F17E
:1023E000180703AA103318685968144603C4083341
:1023F000BB422246F7D1186820609B88A380DDE9A4
:102400000E23CDE900230123ADF808302B6869467F
:10241000DB6B2846984705EB46152B791A075CBFFE
:1024200043F008032B7101E0002AF4D109B0F0BD9C
:102430002DE9F0479A4688B00746884691463023F2
:1024400083F3118807F580546846FFF797FFE06D26
:10245000FFF7AAFD1F282AD9E06D20226946FFF761
:10246000B5FE202823D103AD444605AB2E4603CE4E
:102470009E4220606160354604F10804F6D1306860
:102480002060B388A380DDE90023C9E90023BDF8FB
:102490000830AAF80030002383F3118853464A46D7
:1024A0004146384608B0BDE8F04700F01FBC0020A8
:1024B00080F3118808B0BDE8F08700002DE9F84FDF
:1024C0000023C0E90133254B044640F8183B0F4672
:1024D000FFF74EFF04F12800FFF750FF04F1480812
:1024E00004F582554646083530462036FFF746FF4C
:1024F000AE42F9D104F580554FF480534FF00009F6
:10250000C5E91339C5F848800123EE6504F58758FD
:1025100004F58456C5F8549085F8583085F8603035
:10252000083608F108084FF0000A4FF0000B46E9A2
:1025300008ABA6F11800FFF71BFF203646F8289CD1
:102540004645F4D185F8D07017B1054800F0B8FBC6
:10255000044B63612046BDE8F88F00BFD06C0008D3
:10256000A86C00080064004010B5044B19780446BC
:102570004A1C1A70FFF7A2FF204610BD884B0020AE
:102580002DE9F047002950D0294B2A4FB7FBF1F530
:1025900099428CBF0A231123581EB5FBF3FC03FBA1
:1025A0001C53C4B22BB102280346F5D80020BDE865
:1025B000F0870CF1FF36B6F5806FF7D2C4EBC40E8E
:1025C0000EF103034FEAE309C3F3C703A4EB0308C7
:1025D00009F1010A4FF47A755FFA88F009FB055595
:1025E0005AFA88F8B5FBF8F5B5F5617FC1BF0EF171
:1025F000FF33C3F3C703E01AC0B25C1C50FA84F483
:102600000CFB04F4B7FBF4F4A142CFD1013BDBB2E5
:102610000F2BCBD80138C0B20728C7D800211071C2
:1026200016809170D3700120C1E70846BFE700BF54
:102630003F420F0080DE800270B505460E464FF423
:102640007A746B695B6803F00103B34207D04FF4FF
:102650007A7002F095FB013CF3D1204670BD012059
:10266000FCE7000030B54269936913F0700F16D093
:1026700000230B4C936103F1840200EB42121179A9
:102680004D0709D5890707D5416954F823508D6056
:10269000117941F0040111710133032BEBD130BDED
:1026A000BC6C000873B51D46436916469A68D2078C
:1026B000044609D59A6801219960C2F34002CDE928
:1026C00000650021FFF768FE63699A68D1050BD5A4
:1026D0009A684FF480719960C2F34022CDE9006599
:1026E00001212046FFF758FE63699A68D2030BD593
:1026F0009A684FF480319960C2F34042CDE9006599
:1027000002212046FFF748FE04F58053D3F8CC00A1
:1027100010B103681B699847204602B0BDE87040BD
:10272000FFF7A0BFF8B504464669002972D106F14B
:102730000C073868800770D006EB01153868D5F8AB
:10274000B00110F0040FD5F8B0011ABFC00840F076
:102750000040400DA061D5F8B0C11CF0020F1CBFB5
:1027600040F08040A061D5F8B40106EB011100F003
:102770000F0084F82400D1F8B8012077D1F8B8010F
:10278000000A6077D1F8B801000CA077D1F8B80141
:10279000000EE077D1F8BC0184F82000D1F8BC012C
:1027A000000A84F82100D1F8BC01000C84F8220052
:1027B000D1F8BC11090E84F823103821396004F1D6
:1027C000340004F1180104F1240551F8046B40F8B9
:1027D000046BA942F9D109880180C4E90A23214682
:1027E0000023238651F8283B2046DB6B984704F5ED
:1027F000805393F8C820D3F8CC0042F0040283F849
:10280000C82010B103681B6998472046BDE8F8400E
:10281000FFF728BF06F110078BE7F8BD10B5044697
:1028200000F056FA02460B4652EA030102D0013A82
:1028300063F100030449086820B12146BDE8104057
:10284000FFF770BF10BD00BF844B0020F0B53021F2
:1028500081F31188DFF848C000F583510831002466
:1028600004F1840500EB45152E7977070ED4F606A2
:102870000CD5D1E9007697429E4107D246695CF8B3
:102880002470B7602E7946F004062E710134032CB3
:1028900001F12001E4D1002383F31188F0BD00BFD2
:1028A000BC6C000808B5302383F31188FFF7DAFE0B
:1028B000002383F3118808BDF8B54369054698687D
:1028C00000F0E050B0F1E05F0F4621D0F8B13023C6
:1028D00083F3118805F583541034002606F1840330
:1028E00005EB43131B791A0706D50136032E04F1B5
:1028F0002004F3D1012007E05B07F6D421463846D7
:1029000000F040FA0028F0D1002383F31188F8BDCD
:102910000120FCE708B5302383F3118800F58050CF
:10292000C06DFFF741FB002383F3118843090CBFFF
:102930000120002008BD0000F8B51D4600231370DB
:102940000F4606461446FFF7E5FF80F00100387099
:1029500025B129463046FFF7AFFF2070F8BD0000D3
:102960002DE9B8410C4615461F46804600F0B0F9E7
:102970000B462178024609B9287850B14046FFF746
:1029800065FFFFF78FFF3B462A462146FFF7D4FF3E
:102990000120BDE8B881000070B5302686F31188AB
:1029A000174B1A6C42F000721A641A6A42F00072F5
:1029B0001A621A6A22F000721A62002383F31188E5
:1029C00000F5805494F8C83013F0010516D1A9B170
:1029D00086F311880321132001F0BCFA032114208F
:1029E00001F0B8FA0321152001F0B4FA94F8C830C8
:1029F00043F0010384F8C83085F3118870BD00BF2F
:102A0000003802402DE9F04700F5805588B095F870
:102A1000D030012B04468846164600F28180814F53
:102A200057F823200AB947F82300D7F800A0C4F8C4
:102A30000C802674BAF1000F64D095F8D030012BC9
:102A400070D001212046FFF7A7FF302383F31188C0
:102A50006269136823F0020313606269136843F02C
:102A600001031360636900275F6187F31188012107
:102A70002046FFF7E1FD002800F09580E86DFFF7A4
:102A800081FA04F58359BA4609F108092022002188
:102A90006846FEF717FF02A8FFF76AFCCDF818A0FA
:102AA0006A4609EB07030DF1180E9446BCE80300D3
:102AB000F44518605960624603F10803F5D1DCF86B
:102AC0000000186020379CF804201A71602FDDD1B7
:102AD00095F8C8306FF38203002785F8C8306A463E
:102AE00041462046ADF80070ADF802708DF80470D4
:102AF000FFF746FD636948BB4FF400421A6008B017
:102B0000BDE8F08741F2D80003F0BEFF814610B166
:102B10005146FFF7D3FCC7F80090B9F1000F8CD1F4
:102B20000020ECE7386803681B6B984701460028D3
:102B300087D13868FFF730FF3868036832465B6832
:102B40004146984700287FF47CAFE9E761221A608C
:102B50009DF802309DF803201B06120402F4702237
:102B600003F040731343BDF80020C2F3090213437E
:102B70009DF804201205022E02F4E0020CBF4FF073
:102B800000410021134362690B43D361636913223F
:102B90005A616269136823F00103136039462046C5
:102BA000FFF74AFD08B96369A6E795F8D03093BBF3
:102BB0006169D1F8002242F00102C1F80022616986
:102BC000D1F8002222F47C5222F00E02C1F8002239
:102BD0006169D1F8002242F46062C1F800226269A2
:102BE000C2F814326269C2F80432626941F6FF71B8
:102BF000C2F80C126269C2F840326269C2F844320B
:102C000063690122C3F81C226269D2F8003223F002
:102C10000103C2F8003295F8C83043F0020385F88A
:102C2000C8306CE7844B002008B500F051F850EA3A
:102C30000103024602D0421E61F10001044B1868F4
:102C400010B10B46FFF72EFDBDE8084001F064B857
:102C5000844B002008B50020FFF7E0FDBDE80840E8
:102C600001F05AB808B50120FFF7D8FDBDE80840CB
:102C700001F052B800B59BB0EFF3098168226846B5
:102C8000FEF7FAFDEFF30583014B9B6BFEE700BFF8
:102C900000ED00E008B5FFF7EDFF000000B59BB0C8
:102CA000EFF3098168226846FEF7E6FDEFF305833E
:102CB000014B5B6BFEE700BF00ED00E0FEE70000AC
:102CC0000FB408B5029802F001F8FEE702F08EBCDE
:102CD00002F070BC13B56C4684E80600031D94E84E
:102CE000030083E80500012002B010BD73B58568BC
:102CF000019155B11B885B0707D4D0E900369B6B67
:102D00009847019AC1B23046A847012002B070BD71
:102D1000F0B5866889B005460C465EB1BDF838301E
:102D20005B070AD4D0E900379B6B98472246C1B2B3
:102D30003846B047012009B0F0BD00220023CDE99C
:102D400000230023ADF808300A4603AB01F1080662
:102D5000106851681C4603C40832B2422346F7D1BA
:102D6000106820609288A280FFF7B2FF0423ADF8BC
:102D700008302B68CDE90001DB6B6946284698478F
:102D8000D8E7000030B503680968DD0FB5EBD17FE7
:102D900023F0604421F060424FEAD1700BD0002B49
:102DA000B8BFA40C0029B8BF920C944202D034BF23
:102DB0000120002030BD944205D1C1F38070C3F3DF
:102DC00080738342F6D194422CBF00200120F1E7AA
:102DD0002DE9F041456A15B94162BDE8F0814B68C3
:102DE00023F06047C3F38A464FEAD37EC3F380786B
:102DF00016EA230638BF3E46AC462B465A68BEEB61
:102E0000D27F22F060440AD0002A18DAA40CB4421F
:102E100017D19D420FD10D60DEE71346EEE7A742C2
:102E200007D102F08044C2F3807242450BD054B106
:102E3000EFE708D2EDE7CCF800100B60CDE7B44225
:102E400001D0B442E5D81A689C46002AE5D1196041
:102E5000C3E700002DE9F047089D01F007044FEAA1
:102E6000D508224405F0070500EBD1004FF47F4957
:102E7000944201D1BDE8F08704F0070705F0070A86
:102E800057453E4638BF5646C6F10806111B8E42CE
:102E900028BF0E46E10808EBD50E415C13F80EC0C2
:102EA000B94029FA06F721FA0AF1FFB28CEA0101CA
:102EB00047FA0AF739408CEA010C03F80EC0344493
:102EC0003544D5E780EA0120082341F2210201B20E
:102ED0004000002980B203F1FF33B8BF504013F027
:102EE000FF03F4D17047000038B50C468D18A54299
:102EF00000D138BD14F8011BFFF7E4FFF7E700002D
:102F000042684AB1136843604389818901339BB2A7
:102F10009942438138BF83811046704770B588B0AD
:102F2000202204460D4668460021FEF7CBFC2046D1
:102F30000495FFF7E5FF024658B16B46054608AE1B
:102F40001C4603CCB44228606960234605F108059D
:102F5000F6D1104608B070BD082817D909280CD042
:102F60000A280CD00B280CD00C280CD00D280CD023
:102F70000E2814BF4020302070470C2070471020CE
:102F800070471420704718207047202070470000B9
:102F9000082817D90C280CD910280CD914280CD9BA
:102FA00018280CD920280CD930288CBF0F200E20CF
:102FB0007047092070470A2070470B2070470C208B
:102FC00070470D20704700002DE9F843078C072F4C
:102FD00004461ED9D0E9029800254FF6FF73C5F1CB
:102FE0002006A5F1200029FA05F108FA06F628FACC
:102FF00000F031430143C9B21846FFF763FF0835BB
:10300000402D0346EBD1E1693A46BDE8F843FFF7AE
:103010006BBF4FF6FF70BDE8F883000010B54B683A
:1030200023B9CA8A63F30902CA8210BD04691A6807
:103030001C600361C38A013BC3824A60EFE7000062
:103040002DE9F84F1D46CB8A0F46C3F30901052928
:10305000814692460B4630D00020AAB207F11A04EE
:103060009EB2042E1FFA80F80FD8904503F1010399
:1030700006D3FB8A0A4462F30903FB8201201AE0AB
:103080001AF80060E6540130EAE79045F1D2A1F168
:10309000050B1C237C68BBFBF3F203FB12BB1FFA7E
:1030A0008BF6002C45D14846FFF72AFF044638B975
:1030B00078606FF00200BDE8F88F4FF00008E6E797
:1030C000002606607860ADB24FF0000B454510D980
:1030D0000AEB0803221D13F8011B9155B1B208F148
:1030E00001081B291FFA88F82BD0454506F1010677
:1030F000F1D8FB8AC3F30902154465F30903BCE761
:10310000013292B21C462368002BF9D16B1F0B448D
:103110001C21B3FBF1F301339BB29A42D3D2BBF132
:10312000000FD0D14846FFF7EBFE20B9C4F800B03D
:10313000BFE70122E7E7C0F800B05E462060044622
:10314000C1E74545D5D94846FFF7DAFE08B9206002
:10315000AFE7C0F800B0002620600446B6E70000E4
:103160002DE9F04F2DED028B1C4683B05B69019277
:1031700007468846002B00F09A80238C2BB1E26929
:10318000002A00F09480072B35D807F10C00FFF7D8
:10319000B7FE054638B96FF00205284603B0BDEC0E
:1031A000028BBDE8F08F14220021FEF78BFB228CEE
:1031B000E16905F10800FEF75FFB208C013080B269
:1031C000FFF7E6FEFFF7C8FE013880B22084013029
:1031D00028746369228C1B782A4403F01F0363F070
:1031E0003F0348F000411372384669602946FFF7F3
:1031F000EFFD0125D1E700F10C034FF0000908EEC7
:10320000103A4FF0800A4E464D4618EE100AFFF76E
:1032100077FE83460028BED014220021FEF752FB21
:10322000002E3AD1019BABF8083002220BF1080EB8
:103230001FFA82FC0CF10100BCF1060F218C80B258
:1032400001D88E422BD3FFF7A3FEFFF785FE6269FC
:103250001278013802F01F028E4208BF4FF0400A78
:1032600042EA49121BFA80F14AEA020A013048F0A8
:10327000004281F808A08BF81000CBF804205946D2
:103280003846FFF7A5FD238C0135B3422DB289F0F6
:1032900001094FF0000AB8D17FE70022C6E7E169D3
:1032A000895D0EF802100136B6B20132C0E76FF048
:1032B000010572E7F8B515460E4630220021044696
:1032C0001F46FEF7FFFA069B6360B5F5001F079BDC
:1032D000A76034BF6A094FF6FF72A36297B2E66136
:1032E00004F1100000239A4206D800230360A7824D
:1032F000E3822383E360F8BD066001333046203665
:10330000F1E7000003781BB94BB2002BC8BF017076
:103310007047000000787047F8B50C46C969074649
:1033200011B9238C002B37D1257E1F2D34D8387846
:1033300028BB228C072A2CD8268A36F003032BD1EF
:103340004FF6FF70FFF7D0FD20F00100310240047E
:1033500041EA0561400C41EA40254FF6FF722346E1
:1033600029463846FFF7FCFE002807DD626913781E
:103370000133DBB21F2B88BF00231370F8BD218AF5
:103380002D0645EA012505432046FFF71DFE0246AE
:10339000E5E76FF00300F1E76FF00100EEE70000F2
:1033A00070B58AB0044616460021282268461D469C
:1033B000FEF788FABDF83830ADF810300F9B059352
:1033C0009DF840308DF81830119B07936946BDF881
:1033D0004830ADF820302046CDE90265FFF79CFF6C
:1033E0000AB070BD2DE9F041D36905460C4616467A
:1033F0000BB9138C5BBB377E1F2F28D895F8008044
:10340000B8F1000F26D03046FFF7DEFD33782102F9
:1034100041EAC33141EA0801338A41EA076141EADE
:1034200003410246334641F080012846FFF798FEEB
:1034300000280ADD3378012B07D172691378013334
:10344000DBB21F2B88BF00231370BDE8F0816FF043
:103450000100FAE76FF00300F7E70000F0B58BB06A
:1034600004460D4617460021282268461E46FEF7F0
:1034700029FA9DF84C305A1E534253418DF80030C2
:103480009DF84030ADF81030119B05939DF8483001
:103490008DF81830149B07936A46BDF85430ADF888
:1034A000203029462046CDE90276FFF79BFF0BB07E
:1034B000F0BD0000406A00B104307047436A1A68EA
:1034C000426202691A600361C38A013BC38270478A
:1034D0002DE9F041D0F82080194E14461D46414692
:1034E000002709B9BDE8F081D1E90223A21A65EBF2
:1034F0000303964277EB03031ED2036A8B420DD17E
:10350000FFF78CFD036A1B68036203690B60C38AC3
:103510000161016A013BC3828846E2E7FFF77EFD55
:103520000B68C8F8003003690B60C38A0161013B76
:10353000C382D8F80010D4E788460968D1E700BFF5
:1035400080841E002DE9F04F8BB00D46DDF85090C1
:1035500014469B468046002800F01981B9F1000FFF
:1035600000F01581531E3F2B00F21181012A03D177
:10357000BBF1000F40F00B810023CDE90833B8F810
:103580001430B5EBC30F4FEAC30703D300200BB0D1
:10359000BDE8F08F2B199F42D8F80C303ABF7F1B43
:1035A000FFB227461BB9D8F81030002B7AD0272D50
:1035B0004ED8C5F12806B7424FF000032CBFF6B233
:1035C0003E4600932946D8F8080008AB3246FFF77C
:1035D00041FCA7EB060A35445FFA8AFAB8F81430C2
:1035E00003F10053053BDB000493D8F80C30039340
:1035F0002821039B13B1BAF1000F2CD1D8F8100089
:1036000040B1BAF1000F05D0009608AB5246691AD6
:10361000FFF720FC38B2002FB8D066070AD00AABFB
:1036200003EBD401624211F8083C02F00702134197
:1036300001F8083C082C3CD9102C40F2B580202C15
:1036400040F2B780BBF1000F00F09C80082334E00B
:10365000BA460026C2E7049BE02B28BFE02306936E
:103660000B44AB42059314D95A1B0398009692451C
:1036700034BF5246D2B2691A08AB04300792FFF742
:10368000E9FB079A1644AAEB020A1544F6B25FFA60
:103690008AFA049B069A05999B1A0493039B1B685C
:1036A0000393A6E70093D8F8080008AB3A462946EA
:1036B000AEE7BBF1000F13D00123B4EBC30F6CD006
:1036C000082C12D89DF82030621E23FA02F2D5078A
:1036D00006D54FF0FF3202FA04F423438DF8203070
:1036E0009DF8203089F8003051E7102C12D8BDF831
:1036F0002030621E23FA02F2D10706D54FF0FF32C6
:1037000002FA04F42343ADF82030BDF82030A9F8C4
:1037100000303CE7202C0FD80899631E21FA03F3F0
:10372000DA0705D54FF0FF3202FA04F40C4308948F
:10373000089BC9F800302AE7402C2BD0DDE908654A
:10374000611EC4F12102A4F1210326FA01F105FA58
:1037500002F225FA03F311431943CB0712D50122D4
:10376000A4F12003C4F1200102FA03F322FA01F1CB
:10377000A240524243EA010363EB430332432B432B
:10378000CDE90823DDE90823C9E90023FFE66FF04E
:103790000100FCE66FF00800F9E6082CA0D9102C17
:1037A000B3D9202CEED8C3E7BBF1000FADD0022374
:1037B00083E7BBF1000FBBD004237EE730B5012ABD
:1037C000144638BF0124402C85B028BF4024002572
:1037D000012ACDE9025518D81B788DF80830630707
:1037E0000AD004AB03EBD405624215F8083C02F0A2
:1037F0000702934005F8083C009103462246002149
:1038000002A8FFF727FB05B030BD082AE4D9102A2B
:1038100003D81B88ADF80830E1E7202A8DBFD3E933
:1038200000231B680293CDE90223D8E710B5CB68CB
:103830001BB98B600B618B8210BD04691A681C6018
:103840000361C38A013BC382CA60F0E703064CBF31
:10385000C0F3C0300220704708B50246FFF7F6FFFC
:10386000022806D15306C2F30F2001D100F0030055
:1038700008BDC2F30740FBE72DE9F04F93B0CDE957
:1038800003230A6804461046FFF7E0FF022814BF2E
:10389000C2F306260026002A0D46824680F2F281F7
:1038A00012F0C04940F0EE81097B002900F0EA8166
:1038B000022803D02378B34240F0E781C2F30463C7
:1038C0000693104602F07F030593FFF7C5FF059BA3
:1038D00029444FEA834848EA0A4848EA4668CE78CD
:1038E00000230022CDE90823F309834648EA0008B3
:1038F000029367D0059B009302466768534608A968
:103900002046B847002800F0C381276A4FB94146D6
:1039100004F10C00FFF702FB074690B96FF00200BC
:1039200054E03B6998450DD03F68002FF9D14146DE
:1039300004F10C00FFF7F2FA07460028EED0236AE4
:103940003B60276297F817C006F01F08CCF3840C81
:10395000ACEB08001FFA80FE0028B8BF0EF1200073
:10396000A8EB0C031FFA83FED7E90221B8BF00B20F
:10397000002B0793BEBF0EF120031BB2079352EA40
:10398000010338D0039BDFF824E39A1A049B4FF01D
:10399000000C63EB010196457CEB01032BD36B7BA1
:1039A00097F81AE0734519D1029B002B78D00128B3
:1039B00021DC7868F8B9DFF8F0C2944570EB0103B8
:1039C00016D337E0276A27B96FF00C0013B0BDE8B3
:1039D000F08F3B699845B5D03F68F4E7B248904214
:1039E0007CEB010301D30020F0E7029B002BFAD00F
:1039F000079B0F2B17DCFA7DB30002F0030203F0E4
:103A00007C031343FB7539462046FFF707FB6B7BAE
:103A1000BB76029B3BB9FB7DC3F38402013262F3A8
:103A20008603FB75D0E76A7BBB7E9A42DBD1029BA3
:103A3000002B35D0B309022B32D0039BBB60049B13
:103A4000FB60142200210DA8FDF73CFF039B0A93A5
:103A5000049B0B932B1D0C932B7BADF83EB0013BCD
:103A6000DBB2ADF83C30069B8DF84230059B8DF8FB
:103A7000433094F82C308DF840A083F001038DF88A
:103A800044308DF84180A3680AA920469847FB7D01
:103A9000C3F38403013303F01F039B02FB82A2E7FD
:103AA000FB7DC6F34012B2EBD31F40F0F480C3F3AA
:103AB0008403434540F0F280029A2B7BB609002A2A
:103AC0004DD0F2075DD4032B40F2EB80039BBB602B
:103AD000049BFB602B7BAE1D033BDBB232463946B9
:103AE00004F10C00FFF7ACFA00280CDA3946204646
:103AF000FFF794FAFB7DC3F38403013303F01F0344
:103B00009B02FB820AE7DDE90884AB883B834FF622
:103B1000FF73C9F12000A9F1200228FA09F104FA83
:103B200000F0014324FA02F211431846C9B2FFF72C
:103B3000C9F909F10809B9F1400F0346E9D1B88282
:103B40002A7B033AD2B23146FFF7CEF9FB7DB88229
:103B5000DA43C2F3C01262F3C713FB7543E786B9B9
:103B60002E1D013BDBB23246394604F10C00FFF753
:103B700067FA0028BADB2A7BB88A013AD2B231460A
:103B8000E2E7F98AC1F30901013B0429DAB25BD803
:103B9000281D002307F11B069A4208D910F801CB13
:103BA00006F801C0013101330529DBB2F4D10399D4
:103BB0000A9104990B91934207F11B010C9138BFB4
:103BC000043379680D9134BF55FA83F300230E93C3
:103BD000FB8AADF83EB0C3F309031A44069B8DF887
:103BE0004230059B8DF8433094F82C30ADF83C20E2
:103BF00083F001038DF8443000238DF840A08DF848
:103C000041807B602A7BB88A013A291DFFF76CF955
:103C10003B8BB882834203D1A3680AA92046984708
:103C200020460AA9FFF702FEFB7DBA8AC3F384038C
:103C3000013303F01F039B02FB823B8B9A420CBFB4
:103C400000206FF01000C1E67B68002BAFD005208C
:103C500001E01C3033461E68002EFAD1091A081DF7
:103C60002E1D184401EB090CBCF11B0F5FFA89F300
:103C70009DD89A429BD916F8013B00F8013B09F107
:103C80000109EFE76FF00900A0E66FF00A009DE67A
:103C90006FF00B009AE66FF00D0097E66FF00E00E4
:103CA00094E66FF00F0091E640420F0080841E0002
:103CB000EFF3098305494A6B22F001024A63683336
:103CC00083F30988002383F31188704700EF00E035
:103CD000302080F3118862B60C4B0D4AD96821F46C
:103CE000E0610904090C0A43DA60D3F8FC200949B1
:103CF00042F08072C3F8FC200A6842F001020A60B8
:103D00002022DA7783F82200704700BF00ED00E040
:103D10000003FA05001000E010B5302383F311888A
:103D20000E4B5B6813F4006314D0F1EE103AEFF31E
:103D30000984683C4FF08073E361094BDB6B2366B9
:103D400084F3098800F08CFF10B1064BA36110BD0D
:103D5000054BFBE783F31188F9E700BF00ED00E0B6
:103D600000EF00E03F0300084203000802684368D8
:103D70001143016003B1184770470000024AD3683D
:103D800043F0C003D36070470044004010B5054CB9
:103D9000054A0021204600F087FA044A044BC4E992
:103DA000972310BD904B00207D3D0008004400404B
:103DB00080DE8002234A037C002918BF0A46012BBB
:103DC00030B5C0F868220CD11F4B984209D11F4B67
:103DD000196C41F400311964196E41F4003119660F
:103DE0001B6EB2F904501468D0F86032D0F85C123F
:103DF000002D03EB5403B3FBF4F3BEBF23F0070520
:103E000003F0070343EA450394888B60D38843F0AB
:103E100040030B61138943F001034B6144F40453E5
:103E200043F02C03CB6004F4A05400230B60B4F5E2
:103E3000806F0B684B680CBF7F23FF2380F86432D0
:103E400030BD00BF106D0008904B002000380240CC
:103E50002DE9F041D0F85C62F7683368DA05044672
:103E60009DB20DD5302383F311884FF48061043067
:103E7000FFF77CFF6FF480733360002383F31188B6
:103E8000302383F3118804F1040815F02F033AD18D
:103E900083F31188380615D5290613D5302383F30B
:103EA000118804F1380000F07BF900284EDA08216F
:103EB000201DFFF75BFF4FF67F733B40F36000234D
:103EC00083F311887A0616D56B0614D5302383F355
:103ED0001188D4E913239A420AD1236C43B127F005
:103EE00040073F041021201D3F0CFFF73FFFF76004
:103EF000002383F31188D4F86822D36843B3BDE864
:103F0000F041106918472B0714D015F0080F0CBFAB
:103F100000214FF48071E80748BF41F02001AA0753
:103F200048BF41F040016B0748BF41F08001404667
:103F3000FFF71CFFAD06736805D594F864122046A0
:103F4000194000F0E1F93568ADB29EE77060B6E760
:103F5000BDE8F08100F1604303F561430901C9B296
:103F600083F80013012200F01F039A4043099B00CD
:103F700003F1604303F56143C3F880211A60704781
:103F8000F8B5154682680669AA420B46816938BFB2
:103F90008568761AB54204460BD218462A46FDF7C4
:103FA0006BFCA3692B44A361A3685B1BA360284639
:103FB000F8BD0CD918463246FDF75EFCAF1BE16830
:103FC0003A463044FDF758FCE3683B44EBE71846BB
:103FD0002A46FDF751FCE368E5E700008368934259
:103FE000F7B51546044638BF8568D0E90460361A2F
:103FF000B5420BD22A46FDF73FFC63692B4463614F
:10400000A36828465B1BA36003B0F0BD0DD9324600
:104010000191FDF731FC0199E068AF1B3A4631444C
:10402000FDF72AFCE3683B44E9E72A46FDF724FC58
:10403000E368E4E710B50A440024C361029B84608E
:10404000C0E90000C0E90511C1600261036210BD52
:1040500008B5D0E90532934201D1826882B98268FD
:10406000013282605A1C42611970D0E904329A42CE
:1040700024BFC3684361002100F09EFE002008BDFC
:104080004FF0FF30FBE7000070B5302304460E46CA
:1040900083F31188A568A5B1A368A269013BA36059
:1040A000531CA36115782269934224BFE368A3617E
:1040B000E3690BB120469847002383F31188284613
:1040C00007E03146204600F067FE0028E2DA85F37B
:1040D000118870BD2DE9F74F04460E4617469846E5
:1040E000D0F81C904FF0300A8AF311884FF0000B83
:1040F000154665B12A4631462046FFF741FF034683
:1041000060B94146204600F047FE0028F1D0002368
:1041100083F31188781B03B0BDE8F08FB9F1000F6D
:1041200003D001902046C847019B8BF31188ED1AFC
:104130001E448AF31188DCE7C0E90511C160C36140
:104140001144009B8260C0E9000001610362704776
:10415000F8B504460D461646302383F31188A76848
:10416000A7B1A368013BA36063695A1C62611D701B
:10417000D4E904329A4224BFE3686361E3690BB176
:1041800020469847002080F3118807E031462046FA
:1041900000F002FE0028E2DA87F31188F8BD000083
:1041A000D0E905239A4210B501D182687AB98268B4
:1041B000013282605A1C82611C7803699A4224BFD2
:1041C000C3688361002100F0F7FD204610BD4FF069
:1041D000FF30FBE72DE9F74F04460E461746984699
:1041E000D0F81C904FF0300A8AF311884FF0000B82
:1041F000154665B12A4631462046FFF7EFFE0346D5
:1042000060B94146204600F0C7FD0028F1D00023E8
:1042100083F31188781B03B0BDE8F08FB9F1000F6C
:1042200003D001902046C847019B8BF31188ED1AFB
:104230001E448AF31188DCE7026843681143016079
:1042400003B11847704700001430FFF743BF000068
:104250004FF0FF331430FFF73DBF00003830FFF759
:10426000B9BF00004FF0FF333830FFF7B3BF000095
:104270001430FFF709BF00004FF0FF311430FFF793
:1042800003BF00003830FFF763BF00004FF0FF327C
:104290003830FFF75DBF0000012914BF6FF0130035
:1042A00000207047FFF772BD37B515460E4A026011
:1042B00000224260C0E902220122044602740B4639
:1042C000009000F15C014FF480721430FFF7B2FEF1
:1042D00000942B464FF4807204F5AE7104F138005F
:1042E000FFF72AFF03B030BD246D000810B530235E
:1042F000044683F31188FFF75DFD02232374002039
:1043000080F3118810BD000038B5C36904460D461E
:104310001BB904210844FFF78FFF294604F114005C
:10432000FFF796FE002806DA201D4FF40061BDE875
:104330003840FFF781BF38BD026843681143016010
:1043400003B118477047000013B5446BD4F8943498
:104350001A681178042915D1217C022912D1197902
:10436000128901238B4013420CD101A904F14C00A6
:1043700001F0BCFFD4F89444019B217902462068E7
:1043800000F0D0F902B010BD143001F03FBF0000C2
:104390004FF0FF33143001F039BF00004C3002F011
:1043A00011B800004FF0FF334C3002F00BB80000A2
:1043B000143001F00DBF00004FF0FF31143001F058
:1043C00007BF00004C3001F0DDBF00004FF0FF32AE
:1043D0004C3001F0D7BF00000020704710B5D0F876
:1043E00094341A6811780429044617D1017C0229F3
:1043F00014D15979528901238B4013420ED11430C4
:1044000001F0A0FE024648B1D4F894444FF4807302
:1044100061792068BDE8104000F072B910BD00005D
:10442000406BFFF7DBBF0000704700007FB5124B09
:10443000036000234360C0E90233012502260F4BCD
:10444000057404460290019300F184022946009607
:104450004FF48073143001F051FE094B0294CDE902
:10446000006304F523724FF48073294604F14C0075
:1044700001F018FF04B070BD4C6D00082144000825
:10448000494300080B68302282F311880A7903EB54
:10449000820290614A79093243F822008A7912B186
:1044A00003EB820398610223C0F894140374002084
:1044B00080F311887047000038B5037F044613B1BC
:1044C00090F85430ABB9201D01250221FFF734FFCD
:1044D00004F1140025776FF0010100F079FC84F8F5
:1044E000545004F14C006FF00101BDE8384000F079
:1044F0006FBC38BD10B5012104460430FFF71CFF26
:104500000023237784F8543010BD000038B50446EA
:104510000025143001F00AFE04F14C00257701F06B
:10452000D9FE201D84F854500121FFF705FF2046D5
:10453000BDE83840FFF752BF90F8443003F0600305
:10454000202B07D190F84520212A4FF0000303D8F3
:104550001F2A06D800207047222AFBD1C0E90E335B
:1045600003E0034A82630722C263036401207047A9
:104570002823002037B5D0F894341A68117804291C
:1045800004461AD1017C022917D119791289012315
:104590008B40134211D100F14C05284601F05AFF1F
:1045A00058B101A9284601F0A1FED4F89444019B1A
:1045B00021790246206800F0B5F803B030BD000054
:1045C000F0B500EB810385B09E6904460D46FEB14F
:1045D000302383F3118804EB8507301D0821FFF792
:1045E000ABFEFB685B691B6806F14C001BB10190D8
:1045F00001F08AFE019803A901F078FE024648B155
:10460000039B2946204600F08DF8002383F3118890
:1046100005B0F0BDFB685A691268002AF5D01B8A04
:10462000013B1340F1D104F14402EAE7093138B506
:1046300050F82140DCB1302383F31188D4F894245E
:104640001368527903EB8203DB689B695D6845B1AF
:1046500004216018FFF770FE294604F1140001F0F0
:104660007BFD2046FFF7BAFE002383F3118838BD97
:104670007047000001F0F0B8012303700023C0E987
:104680000133C36183620362C362436203637047A1
:1046900038B50446302383F311880025C0E903555B
:1046A000C0E90555416001F0E7F80223237085F366
:1046B0001188284638BD000070B500EB810305461F
:1046C0005069DA600E46144618B110220021FDF739
:1046D000F9F8A06918B110220021FDF7F3F831466E
:1046E0002846BDE8704001F091B90000826802F0F0
:1046F000011282600022C0E90422826101F012BA34
:10470000F0B400EB81044789E4680125A4698D4079
:104710003D43458123600023A2606360F0BC01F04B
:104720002DBA0000F0B400EB81040789E46801258C
:1047300064698D403D43058123600023A26063606E
:10474000F0BC01F0A7BA000070B5022300250446B2
:104750000370C0E90255C0E90455C564856180F85D
:10476000345001F0EFF863681B6823B129462046F6
:10477000BDE87040184770BD0378052B10B504469E
:104780000AD080F850300523037043681B680BB1D2
:10479000042198470023A36010BD0000017805297B
:1047A00006D190F85020436802701B6803B1184787
:1047B0007047000070B590F83430044613B1002300
:1047C00080F8343004F14402204601F0CDF96368EA
:1047D0009B68B3B994F8443013F0600535D00021DC
:1047E000204601F06DFC0021204601F05FFC63686B
:1047F0001B6813B1062120469847062384F83430FD
:1048000070BD204698470028E4D0B4F84A30E26BE7
:104810009A4288BFE36394F94430E56B002B4FF074
:10482000300380F20381002D00F0F280092284F829
:10483000342083F311880021D4E90E232046FFF7AA
:1048400071FF002383F31188DAE794F8452003F021
:104850007F0343EA022340F20232934200F0C58014
:1048600021D8B3F5807F48D00DD8012B3FD0022B43
:1048700000F09380002BB2D104F14C02A26302221B
:10488000E2632364C1E7B3F5817F00F09B80B3F559
:10489000407FA4D194F84630012BA0D1B4F84C301D
:1048A00043F0020332E0B3F5006F4DD017D8B3F5F3
:1048B000A06F31D0A3F5C063012B90D8636894F842
:1048C00046205E6894F84710B4F848302046B04758
:1048D000002884D04368A3630368E3631AE0B3F558
:1048E000106F36D040F6024293427FF478AF5C4BB3
:1048F000A3630223E3630023C3E794F84630012B4C
:104900007FF46DAFB4F84C3023F00203C4E90E55C8
:10491000A4F84C30256478E7B4F84430B3F5A06FC0
:104920000ED194F8463084F84E30204601F062F8FB
:1049300063681B6813B10121204698470323237045
:104940000023C4E90E339CE704F14F03A363012362
:10495000C3E72378042B10D1302383F3118820463A
:10496000FFF7C4FE85F311880321636884F84F5074
:1049700021701B680BB12046984794F84630002BF5
:10498000DED084F84F300423237063681B68002B4B
:10499000D6D0022120469847D2E794F848301D0629
:1049A00003F00F0120460AD501F0D0F8012804D009
:1049B00002287FF414AF2B4B9AE72B4B98E701F0BA
:1049C000B7F8F3E794F84630002B7FF408AF94F87B
:1049D000483013F00F01B3D01A06204602D501F07B
:1049E00083FBADE701F076FBAAE794F84630002B95
:1049F0007FF4F5AE94F8483013F00F01A0D01B06F9
:104A0000204602D501F05CFB9AE701F04FFB97E7E7
:104A1000142284F8342083F311882B462A46294631
:104A20002046FFF76DFE85F31188E9E65DB115229A
:104A300084F8342083F311880021D4E90E23204622
:104A4000FFF75EFEFDE60B2284F8342083F3118825
:104A50002B462A4629462046FFF764FEE3E700BFBF
:104A60007C6D0008746D0008786D000838B590F80A
:104A700034300446002B3ED0063BDAB20F2A34D83D
:104A80000F2B32D8DFE803F03731310822323131D1
:104A90003131313131313737C56BB0F84A309D4251
:104AA00014D2C3681B8AB5FBF3F203FB12556DB930
:104AB000302383F311882B462A462946FFF732FE1E
:104AC00085F311880A2384F834300EE0142384F827
:104AD0003430302383F3118800231A4619462046C8
:104AE000FFF70EFE002383F3118838BD036C03B17A
:104AF00098470023E7E70021204601F0E1FA002172
:104B0000204601F0D3FA63681B6813B106212046E2
:104B100098470623D7E7000010B590F83430142BDF
:104B2000044629D017D8062B05D001D81BB110BDDB
:104B3000093B022BFBD80021204601F0C1FA0021DD
:104B4000204601F0B3FA63681B6813B106212046C2
:104B50009847062319E0152BE9D10B2380F8343050
:104B6000302383F3118800231A461946FFF7DAFD34
:104B7000002383F31188DAE7C3689B695B68002B25
:104B8000D5D1036C03B19847002384F83430CEE7C5
:104B900000230375826803691B6899689142FBD200
:104BA0005A680360426010605860704700230375C4
:104BB000826803691B6899689142FBD85A68036050
:104BC000426010605860704708B50846302383F390
:104BD00011880B7D032B05D0042B0DD02BB983F34B
:104BE000118808BD8B6900221A604FF0FF33836182
:104BF000FFF7CEFF0023F2E7D1E9003213605A60DD
:104C0000F3E70000FFF7C4BF054BD96808751868C3
:104C100002681A60536001220275D860FBF77ABB04
:104C2000004E002030B50C4BDD684B1C87B00446AD
:104C30000FD02B46094A684600F05EF92046FFF780
:104C4000E3FF009B13B1684600F060F9A86907B064
:104C500030BDFFF7D9FFF9E7004E0020C94B00082F
:104C6000044B1A68DB6890689B68984294BF0020E8
:104C700001207047004E0020084B10B51C68D86812
:104C800022681A60536001222275DC60FFF78EFFF4
:104C900001462046BDE81040FBF73CBB004E00201B
:104CA00038B5074C07490848012300252370656083
:104CB00001F008FC0223237085F3118838BD00BF82
:104CC00068500020846D0008004E002008B572B6C0
:104CD000044B186500F050FC00F006FD024B032267
:104CE0001A70FEE7004E00206850002000F044B922
:104CF000034A516853685B1A9842FBD8704700BF5B
:104D0000001000E08B60022308618B820846704728
:104D10008368A3F1840243F8142C026943F8442CFD
:104D2000426943F8402C094A43F8242CC26843F8EE
:104D3000182C022203F80C2C002203F80B2C044A36
:104D400043F8102CA3F12000704700BF2D0300088A
:104D5000004E002008B5FFF7DBFFBDE80840FFF775
:104D600051BF0000024BDB6898610F20FFF74CBF7A
:104D7000004E0020302383F31188FFF7F3BF0000BB
:104D800008B50146302383F311880820FFF74AFF56
:104D9000002383F3118808BD064BDB6839B14268F4
:104DA00018605A60136043600420FFF73BBF4FF068
:104DB000FF307047004E00200368984206D01A6802
:104DC0000260506099611846FFF71CBF70470000F1
:104DD00038B504460D462068844200D138BD0368CA
:104DE00023605C608561FFF70DFFF4E710B5036891
:104DF0009C68A2420CD85C688A600B604C602160A1
:104E0000596099688A1A9A604FF0FF33836010BD29
:104E10001B68121BECE700000A2938BF0A2170B595
:104E200004460D460A26601901F046FB01F032FBEC
:104E3000041BA54203D8751C2E460446F3E70A2E30
:104E400004D9BDE87040012001F07CBB70BD0000BA
:104E5000F8B5144B0D46D96103F1100141600A2ADF
:104E60001969826038BF0A22016048601861A81879
:104E7000144601F013FB0A2701F00CFB431BA3426D
:104E8000064606D37C1C281901F016FB274635463A
:104E9000F2E70A2F04D9BDE8F840012001F052BB27
:104EA000F8BD00BF004E0020F8B506460D4601F0E3
:104EB000F1FA0F4A134653F8107F9F4206D12A4653
:104EC00001463046BDE8F840FFF7C2BFD169BB6874
:104ED000441A2C1928BF2C46A34202D92946FFF7B1
:104EE0009BFF224631460348BDE8F840FFF77EBFEE
:104EF000004E0020104E002010B4C0E90323002310
:104F00005DF8044B4361FFF7CFBF000010B5194CAB
:104F1000236998420DD0D0E90032816813605A604D
:104F20009A680A449A60002303604FF0FF33A3613C
:104F300010BD2346026843F8102F53600022026020
:104F400022699A4203D1BDE8104001F0AFBA9368DC
:104F500081680B44936001F09DFA2269E1699268CF
:104F6000441AA242E4D91144BDE81040091AFFF7DF
:104F700053BF00BF004E00202DE9F047DFF8BC8092
:104F800008F110072C4ED8F8105001F083FAD8F829
:104F90001C40AA68031B9A423ED81444D5E900324B
:104FA0004FF00009C8F81C4013605A60C5F8009023
:104FB000D8F81030B34201D101F078FA89F31188A2
:104FC000D5E9033128469847302383F311886B696C
:104FD000002BD8D001F05EFA6A69A0EB04094A45BB
:104FE00082460DD2022001F0ADFA0022D8F810302E
:104FF000B34208D151462846BDE8F047FFF728BF25
:10500000121A2244F2E712EB090938BF4A46294630
:105010003846FFF7EBFEB5E7D8F81030B34208D0BA
:105020001444211AC8F81C00A960BDE8F047FFF736
:10503000F3BEBDE8F08700BF104E0020004E0020F8
:1050400038B501F027FA054AD2E90845031B1819BB
:1050500045F10001C2E9080138BD00BF004E002043
:1050600000207047FEE70000704700004FF0FF305F
:105070007047000002290CD0032904D001290748F9
:1050800018BF00207047032A05D8054800EBC2006E
:105090007047044870470020704700BF5C6E0008EE
:1050A00038230020106E000870B59AB005460846F7
:1050B00001A9144600F0C2F801A8FCF7FBFB431C51
:1050C0005B00C5E900340022237003236370C6B27D
:1050D00001AB02341046D1B28E4204F1020401D871
:1050E0001AB070BD13F8011B04F8021C04F8010C7F
:1050F0000132F0E708B5302383F311880348FFF746
:1051000039FA002383F3118808BD00BF70500020D6
:1051100090F8443003F01F02012A07D190F845208F
:105120000B2A03D10023C0E90E3315E003F060031E
:10513000202B08D1B0F848302BB990F84520212A0F
:1051400003D81F2A04D8FFF7F7B9222AEBD0FAE7D1
:10515000034A82630722C26303640120704700BFD1
:105160002F23002007B5052917D8DFE801F019160D
:1051700003191920302383F31188104A019001216B
:10518000FFF79AFA01980E4A0221FFF795FA0D48A7
:10519000FFF7BCF9002383F3118803B05DF804FB2B
:1051A000302383F311880748FFF786F9F2E73023AD
:1051B00083F311880348FFF79DF9EBE7B06D000812
:1051C000D46D00087050002038B50C4D0C4C0D49C2
:1051D0002A4604F10800FFF767FF05F1CA0204F14F
:1051E00010000949FFF760FF05F5CA7204F11800C5
:1051F0000649BDE83840FFF757BF00BF38550020CB
:1052000038230020906D00089A6D0008A56D0008F5
:1052100070B5044608460D46FCF74CFBC6B2204666
:10522000013403780BB9184670BD32462946FCF7A5
:105230002DFB0028F3D10120F6E700002DE9F0470F
:1052400005460C46FCF736FB2C49C6B22846FFF74C
:10525000DFFF08B10836F6B229492846FFF7D8FF24
:1052600008B11036F6B2632E0BD8DFF89080DFF865
:105270009090244FDFF898A02E7846B92670BDE8AC
:10528000F08729462046BDE8F04701F0BBBC252E3B
:1052900030D1072241462846FCF7F8FA80B91A4B6C
:1052A000224603F10C0153F8040B42F8040B8B4225
:1052B000F9D119889B781180937007350F34DBE79B
:1052C000082249462846FCF7E1FA98B90F4BA21C80
:1052D000197809090232C95D02F8041C13F8011B90
:1052E00001F00F015345C95D02F8031CF0D11834D9
:1052F0000835C1E704F8016B0135BDE77C6E000895
:10530000A56D0008846E0008226C0008107AFF1F4B
:105310001C7AFF1FBFF34F8F024AD368DB03FCD414
:10532000704700BF003C024008B5094B1B7873B9B9
:10533000FFF7F0FF074B1A69002ABFBF064A5A6001
:1053400002F188325A601A6822F480621A6008BD3D
:1053500096570020003C02402301674508B50B4BDF
:105360001B7893B9FFF7D6FF094B1A6942F0004248
:105370001A611A6842F480521A601A6822F4805244
:105380001A601A6842F480621A6008BD96570020BD
:10539000003C02401728F0B516D80C4C0C49237875
:1053A0007BB90C4D0E4618234FF0006255F8047B74
:1053B00046F8042B013B13F0FF033A44F6D10123D6
:1053C000237051F82000F0BD0020FCE7F8570020C2
:1053D00098570020986E0008014B53F82000704742
:1053E000986E000818207047172810B5044601D998
:1053F000002010BDFFF7CEFF064B53F824301844B1
:10540000C21A0BB90120F4E712680132F0D1043B53
:10541000F6E700BF986E0008172838B5044628D86C
:105420001549FFF777FFFFF77FFFF323CB600C23CE
:10543000B0FBF3F203FB1205D30143EAC503DBB271
:1054400043F4007343F002030B610B6943F48033B0
:105450000B61FFF75FFFFFF79DFF084B53F8241028
:1054600000F03EF9FFF77AFF2046BDE83840FFF72D
:10547000BBBF002038BD00BF003C0240986E000852
:10548000F8B512F00103144642D18218B2F1026F4E
:1054900057D82D4B1B6813F0010352D02B4DFFF74B
:1054A00043FFF323EB60FFF735FF40F20127032CA6
:1054B00015D824F001046618244C401A40F2011754
:1054C000B142236900EB010524D123F001032361DC
:1054D000FFF744FF0120F8BD043C0430E7E78307F1
:1054E000E7D12B6923F440732B612B693B432B617C
:1054F00051F8046B0660BFF34F8FFFF70BFF036893
:105500009E42E9D02B6923F001032B61FFF726FFB0
:105510000020E0E723F44073236123693B432361C8
:105520000B882B80BFF34F8FFFF7F4FE2D8831F8E7
:10553000023BADB2AB42C3D0236923F00103236128
:10554000E4E71846C7E700BF00380240003C0240CD
:10555000084908B50B7828B11BB9FFF7E5FE012310
:105560000B7008BD002BFCD0BDE808400870FFF7A9
:10557000F5BE00BF9657002008B50649064800F062
:10558000B1F8BDE808404FF480314FF0805000F092
:10559000A9B800BF00FF0200000100200846114624
:1055A00001F094BA012001F091BA0000084601F020
:1055B000ABBA000038B5EFF311859DB9EFF3058460
:1055C000C4F30804302334B183F31188FFF738FDA6
:1055D00085F3118838BD83F31188FFF731FD84F31B
:1055E000118838BDBDE83840FFF72ABD38B5FFF750
:1055F000E1FF114C114AC00840EA4170A0FB025E75
:10560000C908A0FB040C1CEB050CA1FB04404FF0E7
:1056100000035B41A1FB02121CEB040C43EB0000F6
:1056200011EB0E0142F10002411842F1000009099C
:1056300041EA007038BD00BFCFF753E3A59BC420FB
:1056400010B50244064BD2B2904200D110BD441CAA
:1056500000B253F8200041F8040BE0B2F4E700BFB9
:10566000502800400F4B30B51C6F240407D41C6F2A
:1056700044F400741C671C6F44F400441C670A4C1B
:10568000236843F4807323600244084BD2B29042F3
:1056900000D130BD441C00B251F8045B43F82050E7
:1056A000E0B2F4E7003802400070004050280040AB
:1056B00007B5012201A90020FFF7C2FF019803B03E
:1056C0005DF804FB13B50446FFF7F2FFA04205D0D6
:1056D000012201A900200194FFF7C4FF02B010BD10
:1056E000704700007047000070470000094B5A885F
:1056F000B2F5805F10460BD022F0020341F20102A6
:10570000934205D041F20703C31A584258417047EB
:1057100001207047002004E0074B45F255521A6003
:1057200002225A6040F6FF729A604CF6CC421A6030
:10573000024B01221A7070470030004000580020D0
:10574000034B1B781BB1034B4AF6AA221A60704721
:105750000058002000300040034B1A681AB9034A71
:10576000D2F874281A607047FC57002000300240BD
:10577000024B4FF08072C3F874287047003002402B
:1057800008B5FFF7E9FF024B1868C0F3407008BD89
:10579000FC57002008B5FFF7DFFF024B1868C0F385
:1057A000007008BDFC57002070470000FEE70000B5
:1057B0000A4B0B480B4A90420BD30B4BDA1C121AC4
:1057C000C11E22F003028B4238BF00220021FCF7E9
:1057D00079B853F8041B40F8041BECE7EC700008A0
:1057E00004590020045900200459002070B5D0E964
:1057F00015439E6800224FF0FF3504EB4213510120
:10580000D3F800090028BEBFD3F8000940F080405B
:10581000C3F80009D3F8000B0028BEBFD3F8000B73
:1058200040F08040C3F8000B013263189642C3F881
:105830000859C3F8085BE0D24FF00113C4F81C38D4
:1058400070BD0000890141F02001016103699B06E0
:10585000FCD41220FFF74CBA10B5054C2046FEF7D9
:105860000BFF4FF0A0436365024BA36510BD00BF63
:10587000045800201C6F000870B50378012B054602
:1058800050D12A4B446D98421BD1294B5A6B42F0A0
:1058900080025A635A6D42F080025A655A6D5A6905
:1058A00042F080025A615A6922F080025A610E2148
:1058B00043205B69FEF74EFB1E4BE3601E4BC4F8B2
:1058C00000380023C4F8003EC02323606E6D4FF4FF
:1058D0005023A3633369002BFCDA012333610C20CE
:1058E000FFF706FA3369DB07FCD41220FFF700FA52
:1058F0003369002BFCDA0026A6602846FFF776FF06
:105900006B68C4F81068DB68C4F81468C4F81C68D5
:105910004BB90A4BA3614FF0FF336361A36843F0B7
:105920000103A36070BD064BF4E700BF04580020DC
:10593000003802404014004003002002003C30C008
:10594000083C30C0F8B5446D054600212046FFF7FD
:1059500079FFA96D00234FF001128F68C4F8343825
:105960004FF00066C4F81C284FF0FF3004EB4312E0
:1059700001339F42C2F80069C2F8006BC2F80809FF
:10598000C2F8080BF2D20B686A6DEB6563621023F4
:105990001361166916F01006FBD11220FFF7A8F963
:1059A000D4F8003823F4FE63C4F80038A36943F444
:1059B000402343F01003A3610923C4F81038C4F84E
:1059C00014380A4BEB604FF0C043C4F8103B084B4F
:1059D000C4F8003BC4F81069C4F80039EB6D03F15A
:1059E000100243F48013EA65A362F8BDF86E000864
:1059F00040800010426D90F84E10D2F8003823F429
:105A0000FE6343EA0113C2F8003870472DE9F843FA
:105A100000EB8103456DDA68166806F00306731E15
:105A2000022B05EB41130C4680460FFA81F94FEA31
:105A300041104FF00001C3F8101B4FF0010104F1B9
:105A4000100398BFB60401FA03F391698EBF334E79
:105A500006F1805606F5004600293AD0578A04F12F
:105A60005801490137436F50D5F81C180B43C5F84E
:105A70001C382B180021C3F8101953690127611E27
:105A8000A7409BB3138A928B9B08012A88BF53437C
:105A9000D8F85C20981842EA034301F1400205EB74
:105AA0008202C8F85C00214653602846FFF7CAFE10
:105AB00008EB8900C3681B8A43EA845348346401B5
:105AC0001E432E51D5F81C381F43C5F81C78BDE87D
:105AD000F88305EB4917D7F8001B21F40041C7F8FC
:105AE000001BD5F81C1821EA0303C0E704F13F03AB
:105AF00005EB83030A4A5A6028462146FFF7A2FEB7
:105B000005EB4910D0F8003923F40043C0F8003900
:105B1000D5F81C3823EA0707D7E700BF008000103C
:105B200000040002826D1268C265FFF75FBE0000CC
:105B30005831436D49015B5813F4004004D013F40D
:105B4000001F0CBF02200120704700004831436D48
:105B500049015B5813F4004004D013F4001F0CBF3C
:105B6000022001207047000000EB8101CB68196A18
:105B70000B6813604B6853607047000000EB8103B3
:105B800030B5DD68AA691368D36019B9402B84BFAA
:105B9000402313606B8A1468426D1C44013CB4FBC3
:105BA000F3F46343033323F0030302EB411043EAAE
:105BB000C44343F0C043C0F8103B2B6803F0030319
:105BC000012B09B20ED1D2F8083802EB411013F4C0
:105BD000807FD0F8003B14BF43F0805343F0005364
:105BE000C0F8003B02EB4112D2F8003B43F0044303
:105BF000C2F8003B30BD00002DE9F041244D6E6D30
:105C000006EB40130446D3F8087BC3F8087B38073B
:105C10000AD5D6F81438190706D505EB84032146B2
:105C2000DB6828465B689847FA071FD5D6F8143812
:105C3000DB071BD505EB8403D968CCB98B69488A8F
:105C40005A68B2FBF0F600FB16228AB91868DA68C7
:105C500090420DD2121AC3E90024302383F3118835
:105C60000B482146FFF78AFF84F31188BDE8F081D5
:105C7000012303FA04F26B8923EA02036B81CB68E8
:105C8000002BF3D021460248BDE8F041184700BF81
:105C90000458002000EB810370B5DD68436D6C692A
:105CA0002668E6604A0156BB1A444FF40020C2F849
:105CB00010092A6802F00302012A0AB20ED1D3F8B1
:105CC000080803EB421410F4807FD4F8000914BFD5
:105CD00040F0805040F00050C4F8000903EB42123D
:105CE000D2F8000940F00440C2F80009D3F83408A3
:105CF000012202FA01F10143C3F8341870BD19B949
:105D0000402E84BF4020206020682E8A8419013CE8
:105D1000B4FBF6F440EAC44040F000501A44C6E731
:105D20002DE9F8433B4D6E6D06EB40130446D3F866
:105D30000889C3F8088918F0010F4FEA40171AD0F4
:105D4000D6F81038DB0716D505EB8003D9684B6908
:105D50001868DA68904230D2121A4FF000091A60BF
:105D6000C3F80490302383F3118821462846FFF7B7
:105D700091FF89F3118818F0800F1CD0D6F83438C1
:105D80000126A640334216D005EB84036D6DD3F88F
:105D90000CC0DCF814200134E4B2D2F800E005EBCA
:105DA00004342F445168714515D3D5F8343823EAAB
:105DB0000606C5F83468BDE8F883012303FA04F247
:105DC0002B8923EA02032B818B68002BD3D0214639
:105DD00028469847CFE7BCF81000AEEB010383429A
:105DE00028BF0346D7F8180980B2B3EB800FE2D87A
:105DF0009068A0F1040959F8048FC4F80080A0EB62
:105E000009089844B8F1040FF5D818440B44906081
:105E10005360C7E7045800202DE9F74FA24C656D89
:105E20006E69AB691E4016F480586E6107D020463B
:105E3000FEF78AFC03B0BDE8F04FFDF76DBF002E02
:105E400012DAD5F8003E98489B071EBFD5F8003EF1
:105E500023F00303C5F8003ED5F8043823F001030E
:105E6000C5F80438FEF79AFC370505D58E48FFF7CC
:105E7000BDFC8D48FEF780FCB0040CD5D5F8083881
:105E800013F0060FEB6823F470530CBF43F4105368
:105E900043F4A053EB6031071BD56368DB681BB983
:105EA000AB6923F00803AB612378052B0CD1D5F83F
:105EB000003E7D489A071EBFD5F8003E23F003033D
:105EC000C5F8003EFEF76AFC6368DB680BB17648F4
:105ED0009847F30274D4B70227D5D4F85490DFF86A
:105EE000C8B100274FF0010A09EB4712D2F8003B76
:105EF00003F44023B3F5802F11D1D2F8003B002BDF
:105F00000DDA62890AFA07F322EA0303638104EBDC
:105F10008703DB68DB6813B1394658469847A36DA1
:105F200001379B68FFB29F42DED9F00617D5676D37
:105F30003A6AC2F30A1002F00F0302F4F012B2F54B
:105F4000802F00F08580B2F5402F08D104EB830349
:105F50000022DB681B6A07F5805790426AD1300344
:105F6000D5F8184813D5E10302D50020FFF744FE09
:105F7000A20302D50120FFF73FFE630302D50220F2
:105F8000FFF73AFE270302D50320FFF735FE75031E
:105F90007FF550AFE00702D50020FFF7C1FEA10753
:105FA00002D50120FFF7BCFE620702D50220FFF7F1
:105FB000B7FE23077FF53EAF0320FFF7B1FE39E7B9
:105FC000636DDFF8E4A0019300274FF00109A36D92
:105FD0009B685FFA87FB9B453FF67DAF019B03EB18
:105FE0004B13D3F8001901F44021B1F5802F1FD1D4
:105FF000D3F8001900291BDAD3F8001941F09041B9
:10600000C3F80019D3F800190029FBDB5946606D6D
:10601000FFF718FC218909FA0BF321EA0303238116
:1060200004EB8B03DB689B6813B1594650469847D5
:106030000137CCE7910708BFD7F80080072A98BF3F
:1060400003F8018B02F1010298BF4FEA182884E798
:10605000023304EB830207F580575268D2F818C068
:10606000DCF80820DCE9001CA1EB0C0C00218842C4
:106070000AD104EB830463689B699A6802449A60BE
:106080005A6802445A606AE711F0030F08BFD7F854
:1060900000808C4588BF02F8018B01F1010188BFA7
:1060A0004FEA1828E3E700BF04580020436D03EBD4
:1060B0004111D1F8003B43F40013C1F8003B704795
:1060C000436D03EB4111D1F8003943F40013C1F8DB
:1060D00000397047436D03EB4111D1F8003B23F4C5
:1060E0000013C1F8003B7047436D03EB4111D1F839
:1060F000003923F40013C1F80039704730B5039C10
:106100000172043304FB0325C0E90653049B0363B7
:106110000021059BC160C0E90000C0E90422C0E97C
:106120000842C0E90A11436330BD0000416A002201
:10613000C0E90411C0E90A22C2606FF00101FEF754
:1061400047BE0000D0E90432934201D1C2680AB9C7
:10615000181D70470020704703691960C26801323A
:10616000C260C269134482690361934224BF436AD7
:1061700003610021FEF720BE38B504460D46E368F2
:106180003BB16269131D1268A3621344E3620020ED
:1061900007E0237A33B929462046FEF7FDFD0028A3
:1061A000EDDA38BD6FF00100FBE70000C368C2699B
:1061B000013BC3604369134482694361934224BF36
:1061C000436A436100238362036B03B1184770473E
:1061D00070B53023044683F31188866A3EB9FFF711
:1061E000CBFF054618B186F31188284670BDA36A17
:1061F000E26A13F8015BA362934202D32046FFF7E1
:10620000D5FF002383F31188EFE700002DE9F84F55
:1062100004460E46174698464FF0300989F3118818
:106220000025AA46D4F828B0BBF1000F09D1414699
:106230002046FFF7A1FF20B18BF311882846BDE867
:10624000F88FD4E90A12A7EB050B521A934528BF21
:106250009346BBF1400F1BD9334601F1400251F880
:10626000040B43F8040B9142F9D1A36A4033403642
:10627000A3624035D4E90A239A4202D32046FFF7AD
:1062800095FF8AF31188BD42D8D289F31188C9E7F6
:1062900030465A46FBF7F0FAA36A5B445E44A362B9
:1062A0005D44E7E710B5029C0172043303FB04214F
:1062B000C0E906130023C0E90A33039B0363049B70
:1062C000C460C0E90000C0E90422C0E90842436399
:1062D00010BD0000026AC260426AC0E904220022C6
:1062E000C0E90A226FF00101FEF772BDD0E9042374
:1062F0009A4201D1C26822B9184650F8043B0B609B
:10630000704700231846FAE7C368C2690133C360C7
:106310004369134482694361934224BF436A4361E2
:106320000021FEF749BD000038B504460D46E3687C
:106330003BB123691A1DA262E2691344E3620020A3
:1063400007E0237A33B929462046FEF725FD0028C9
:10635000EDDA38BD6FF00100FBE70000036919605A
:10636000C268013AC260C269134482690361934200
:1063700024BF436A036100238362036B03B11847A0
:106380007047000070B530230D460446114683F374
:106390001188866A2EB9FFF7C7FF10B186F31188FE
:1063A00070BDA36A1D70A36AE26A01339342A362BF
:1063B00004D3E16920460439FFF7D0FF002080F3C1
:1063C0001188EDE72DE9F84F04460D4690469946B1
:1063D0004FF0300A8AF311880026B346A76A4FB9F6
:1063E00049462046FFF7A0FF20B187F311883046C9
:1063F000BDE8F88FD4E90A073A1AA8EB06079742D6
:1064000028BF1746402F1BD905F1400355F8042B30
:1064100040F8042B9D42F9D1A36A4033A362403671
:10642000D4E90A239A4204D3E16920460439FFF7EC
:1064300095FF8BF311884645D9D28AF31188CDE7B1
:1064400029463A46FBF718FAA36A3B443D44A36247
:106450003E44E5E7D0E904239A4217D1C3689BB1D3
:10646000836A8BB1043B9B1A0ED01360C368013B57
:10647000C360C3691A44836902619A4224BF436AB4
:106480000361002383620123184670470023FBE762
:1064900000F0D2B84FF08043586A70474FF0804305
:1064A000002258631A610222DA6070474FF080437D
:1064B0000022DA60704700004FF080435863704755
:1064C000FEE7000070B51B4B01630025044686B053
:1064D000586085620E46FDF7FBFB04F11003C4E92A
:1064E00004334FF0FF33C4E90635C4E90044A56026
:1064F000E562FFF7CFFF2B460246C4E9082304F10B
:1065000034010D4A256580232046FEF7FBFB01235D
:10651000E0600A4A0375009272680192B268CDE9A0
:106520000223074B6846CDE90435FEF713FC06B09D
:1065300070BD00BF68500020286F00082D6F000854
:10654000C1640008024AD36A1843D062704700BF92
:10655000004E00204B6843608B688360CB68C3604B
:106560000B6943614B6903628B6943620B6803608B
:106570007047000008B5264B26481A6940F2FF1103
:106580000A431A611A6922F4FF7222F001021A61A9
:106590001A691A6B0A431A631A6D0A431A651E4A6E
:1065A0001B6D1146FFF7D6FF02F11C0100F580605C
:1065B000FFF7D0FF02F1380100F58060FFF7CAFF56
:1065C00002F1540100F58060FFF7C4FF02F1700191
:1065D00000F58060FFF7BEFF02F18C0100F58060DE
:1065E000FFF7B8FF02F1A80100F58060FFF7B2FFE6
:1065F00002F1C40100F58060FFF7ACFF02F1E00199
:1066000000F58060FFF7A6FFBDE8084000F090B8F5
:106610000038024000000240346F000808B500F066
:106620000BFAFEF73DFBFFF797F8BDE80840FEF7D1
:10663000CBBD0000704700000F4B1A6C42F0010206
:106640001A641A6E42F001021A660C4A1B6E9368B5
:1066500043F0010393604FF0804353229A624FF05E
:10666000FF32DA6200229A615A63DA605A600122CC
:106670005A611A60704700BF00380240002004E0F1
:106680004FF0804208B51169D3680B40D9B2C943B5
:106690009B07116107D5302383F31188FEF726FB92
:1066A000002383F3118808BD1F4B1A696FEAC25299
:1066B0006FEAD2521A611A69C2F308021A614FF0E6
:1066C000FF301A695A69586100215A6959615A693B
:1066D0001A6A62F080521A621A6A02F080521A62D2
:1066E0001A6A5A6A58625A6A59625A6A1A6C42F0AD
:1066F00080521A641A6E42F080521A661A6E0B4A61
:10670000106840F480701060186F00F44070B0F5AD
:10671000007F1EBF4FF4803018671967536823F459
:106720000073536000F060B9003802400070004010
:10673000344B4FF080521A64334A4FF44041116099
:106740001A6842F001021A601A689107FCD59A682B
:1067500022F003029A602B4B9A6812F00C02FBD1D4
:10676000196801F0F90119609A601A6842F48032E0
:106770001A601A689203FCD55A6F42F001025A67F8
:10678000204B5A6F9007FCD5204A5A601A6842F095
:1067900080721A601C4A53685904FCD5194B1A6858
:1067A0009201FCD51A4A9A600322C3F88C20194B37
:1067B0001A68194B9A42194B21D1194A1168194A82
:1067C00091421CD140F205121A60144A136803F07A
:1067D0000F03052BFAD10B4B9A6842F002029A6024
:1067E0009A6802F00C02082AFAD15A6C42F48042EC
:1067F0005A645A6E42F480425A665B6E704740F2A9
:106800000572E1E70038024000700040185440076C
:1068100000948838002004E011640020003C02400D
:1068200000ED00E041C20F41074A08B5536903F08B
:106830000103536123B1054A13680BB150689847AF
:10684000BDE80840FDF768BA003C01407C580020D4
:10685000074A08B5536903F00203536123B1054A9F
:1068600093680BB1D0689847BDE80840FDF754BA6B
:10687000003C01407C580020074A08B5536903F0EA
:106880000403536123B1054A13690BB1506998475A
:10689000BDE80840FDF740BA003C01407C580020AC
:1068A000074A08B5536903F00803536123B1054A49
:1068B00093690BB1D0699847BDE80840FDF72CBA41
:1068C000003C01407C580020074A08B5536903F09A
:1068D0001003536123B1054A136A0BB1506A9847FC
:1068E000BDE80840FDF718BA003C01407C58002084
:1068F000164B10B55C6904F478725A61A30604D58E
:10690000134A936A0BB1D06A9847600604D5104ABF
:10691000136B0BB1506B9847210604D50C4A936B4F
:106920000BB1D06B9847E20504D5094A136C0BB143
:10693000506C9847A30504D5054A936C0BB1D06CF5
:106940009847BDE81040FDF7E7B900BF003C0140A3
:106950007C580020194B10B55C6904F47C425A61E4
:10696000620504D5164A136D0BB1506D9847230587
:1069700004D5134A936D0BB1D06D9847E00404D54C
:106980000F4A136E0BB1506E9847A10404D50C4A00
:10699000936E0BB1D06E9847620404D5084A136F0A
:1069A0000BB1506F9847230404D5054A936F0BB180
:1069B000D06F9847BDE81040FDF7AEB9003C0140EC
:1069C0007C58002008B50348FDF742FABDE80840AE
:1069D000FDF7A2B9904B002008B5FFF751FEBDE8C6
:1069E0000840FDF799B90000062108B50846FDF7F3
:1069F000B1FA06210720FDF7ADFA06210820FDF7C0
:106A0000A9FA06210920FDF7A5FA06210A20FDF7BB
:106A1000A1FA06211720FDF79DFA06212820FDF78F
:106A200099FA07211C20FDF795FABDE808400C21D2
:106A30002620FDF78FBA000008B5FFF735FE00F0FD
:106A40000DF8FDF72FFCFDF715FEFDF7EDFCFFF748
:106A5000F1FDBDE80840FFF71BBD00000023054A1B
:106A600019460133102BC2E9001102F10802F8D1D6
:106A7000704700BF7C5800200B460146184600F0C6
:106A80002DB8000000F040B8012838BF012010B533
:106A90000446204600F030F830B900F007F808B995
:106AA00000F00CF88047F4E710BD0000024B1868B6
:106AB000BFF35B8F704700BFFC58002008B506206D
:106AC00000F084F80120FEF7CDFA0000024B0A46E0
:106AD00001461868FEF762BD5823002010B5054C2A
:106AE00013462CB10A4601460220AFF3008010BDC8
:106AF0002046FCE700000000024B01461868FEF744
:106B000051BD00BF58230020024B01461868FEF714
:106B10004DBD00BF5823002010B5013902449042FA
:106B200001D1002005E0037811F8014FA34201D004
:106B3000181B10BD0130F2E72DE9F041A3B1C91ACD
:106B400017780144044603F1FF3C8C42204601D9EA
:106B5000002009E00578BD4204F10104F5D10CEBF9
:106B60000405D618A54201D1BDE8F08115F8018DC4
:106B700016F801EDF045F5D0E7E700001F2938B51C
:106B800004460D4604D9162303604FF0FF3038BD8C
:106B9000426C12B152F821304BB9204600F030F867
:106BA0002A4601462046BDE8384000F017B8012BC0
:106BB0000AD0591C03D1162303600120E7E7002403
:106BC00042F82540284698470020E0E7024B01465E
:106BD0001868FFF7D3BF00BF5823002038B5074D12
:106BE00000230446084611462B60FEF73FFA431C7B
:106BF00002D12B6803B1236038BD00BF00590020CB
:106C0000FEF72EBA034611F8012B03F8012B002AD8
:106C1000F9D170476F72672E6172647570696C6F1D
:106C2000742E50697872616365722D706572697037
:106C30006800000053544D3332463F3F3F005354E9
:106C40004D3332463430780053544D33324634326B
:106C5000780053544D3332463434365858000000CF
:106C6000012033000010410001105A0003105900A8
:106C70000710310000000000346C0008130400000D
:106C80003E6C000819040000486C00082104000054
:106C9000526C000840A2E4F1646891060041A3E54B
:106CA000F2656992070000004261642043414E4949
:106CB0006661636520696E6465782E00800000005F
:106CC00000800000000080000000000000000000C4
:106CD000E5210008052A000861290008252200088E
:106CE0003122000831240008F5210008052200089F
:106CF000F921000801220008FD21000855230008A1
:106D000009220008D52C00081922000829230008B0
:106D100000960000000000000000000000000000DD
:106D20000000000000000000654200085142000819
:106D30008D4200087942000885420008714200082F
:106D40005D42000849420008994200080000000026
:106D5000A543000891430008CD430008B94300084B
:106D6000C5430008B14300089D430008894300085B
:106D7000D9430008000000000100000000000000EE
:106D800063300000806D0008584E002068500020DD
:106D90004172647550696C6F740025424F415244D2
:106DA000252D424C002553455249414C25000000F9
:106DB0000200000000000000C14500082D46000848
:106DC0004000400008550020185500200200000037
:106DD00000000000030000000000000071460008F1
:106DE00000000000100000002855002000000000F6
:106DF0000100000000000000045800200101020012
:106E0000655100087550000811510008F550000840
:106E100043000000186E000809024300020100C090
:106E200032090400000102020100052400100105DE
:106E30002401000104240202052406000107058242
:106E4000030800FF09040100020A00000007050111
:106E5000024000000705810240000000120000000F
:106E6000646E00081201100102000040091241572F
:106E700000020102030100000403090425424F41FE
:106E800052442500303132333435363738394142B7
:106E90004344454600000000004000000040000060
:106EA000004000000040000000000100000002005F
:106EB00000000200000002000000020000000200CA
:106EC000000002000000020000400000004000003E
:106ED000004000000040000000000100000002002F
:106EE000000002000000020000000200000002009A
:106EF000000002000000020000000000B54700088A
:106F00006D4A0008194B00084000400064580020FA
:106F10006458002001000000745800208000000028
:106F200040010000030000006D61696E0069646C3F
:106F3000650000000000802A00000000AAAAAAAA9A
:106F400000000024FFFF00000000000000A00A0075
:106F50004400000000000000AAAAAAAA0000000045
:106F6000FFFF0000000000000000000010000040D3
:106F700000000000AAAAAAAA10000040FFFF00001B
:106F800000000000000000000A681000000000007F
:106F9000AAAAAAAA00541000FFFF000099007007D7
:106FA000000000000000004000000000AAAAAAAAF9
:106FB00000000040FFFF0000000000000000000093
:106FC0000000000000000000AAAAAAAA0000000019
:106FD000FFFF0000000000000000000000000000B3
:106FE00000000000AAAAAAAA00000000FFFF0000FB
:106FF0000000000000000000000000000000000091
:107000000A00000000000000030000000000000073
:107010000000000000000000000000000000000070
:107020000000000000000000000000000000000060
:107030007A0500000000000000001F0000000000B2
:1070400040420F00FE2A0100D2040000FF000000B1
:1070500070500020904B00200096000000000800B7
:10706000960000000008000004000000786E000890
:107070000000000000000000000000000000000010
:1070800000000000000000005C2300200000000061
:1070900000000000000000000000000000000000F0
:1070A00000000000000000000000000000000000E0
:1070B00000000000000000000000000000000000D0
:1070C00000000000000000000000000000000000C0
:1070D00000000000000000000000000000000000B0
:0C70E000000000000000000000000000A4
:00000001FF
